:020000040800F2
:1000000068240020D9000008A9180008A1010008F0
:1000100000000000000000000000000000000000E0
:10002000000000000000000000000000E5000008E3
:1000300000000000000000001F010008731D000800
:10004000EB000008EB000008ED180008EB000008CA
:10005000EB000008EB000008EB000008EB000008D4
:10006000EB000008D10800082D090008000000007E
:10007000EB0000080000000000000000EB0000089A
:10008000EB000008EB000008EB000008EB000008A4
:10009000EB000008EB00000800000000EB00000887
:1000A000EB000008B91F0008EB000008EB00000897
:1000B000F5160008EB000008EB000008EB00000854
:1000C0000448854600F0A0F900F012F90048004706
:1000D00005050008682400200448804704480047BC
:1000E000FEE7FEE7FEE7FEE7FEE7FEE7091E000883
:1000F000C1000008EFF3108072B6704780F31088DB
:1001000070472A4A1368012B03D001231360284A41
:100110001060284A11602848284901607047EFF3B1
:10012000108272B62148016800291DD000210160AB
:100130001F48016800290AD0EFF3098120390068BF
:100140000160F0C144464D4656465F46F0C119492C
:1001500009680968F0C9F0B4F0C9A046A946B246DA
:10016000BB46F0BC81F3098882F31088042040422A
:100170000047104908600E49002008600B49012023
:1001800008600F480F490268114301600A480B4993
:1001900001600D480068006880F3088862B6704707
:1001A000EFF3098000B504F0C7F900BD201300206B
:1001B000F80F0020FC0F002004ED00E0000000100C
:1001C00020ED00E00000FFFF08ED00E0F0B51FB4F7
:1001D0000646002082B005464024019100901BE0B5
:1001E000019922460F46304600F0C5F8049A059B57
:1001F000801A994110D310461946224600F0ABF8F8
:10020000361A8F410197224601200021009F00F0FD
:10021000A2F838184D4100902046641E0028DFDC0B
:10022000019B00982946324607B0F0BD03460B43B8
:100230009B0703D009E008C9121F08C0042AFAD29C
:1002400003E00B780370401C491C521EF9D2704722
:10025000D2B201E00270401C491EFBD2704700225E
:10026000F6E710B513460A4604461946FFF7F0FFB5
:10027000204610BD10B5044605E00B780370401C05
:10028000002B00D0491C521EF7D2204610BD421C44
:100290000178401C0029FBD1801A704730B5044614
:1002A0000020034600E05B1C934203D2E05CCD5C7F
:1002B000401BF8D030BD30B505460020034600E0B5
:1002C0005B1C934205D2EC5CC85C201A01D1002C67
:1002D000F6D130BD70B5064606F076FF04680546D7
:1002E0000A220021304600F057F82C6070BD000053
:1002F0007CB507480090074801900546009C04E043
:100300002046016808188047241DAC42F8D17CBD06
:10031000F4870008F887000870B50446002903D068
:1003200000202022012310E0002801D00020C0433B
:10033000C046C0460DE02546D5408D4205D30D464A
:100340009540641B1D46954040191546521E002DD0
:10035000F1DC214670BD10B5202A04DB0146203AAD
:100360009140002010BD914020239C1A0346E34099
:100370001943904010BD10B5202A04DB0846203AEE
:10038000D040002110BD0B46D340D0402024A21AFB
:1003900091400843194610BDF7B5009C0F46002652
:1003A0002578641C002D05D000F046F80068405DFB
:1003B000C007F5D12B2D02D02D2D18D0641E394643
:1003C0002046029A00F03CF8002F04D03968A14280
:1003D00001D1009939607105022400290BDA4042ED
:1003E000002803DD06F0F0FE0460A007FEBD01203A
:1003F00080020643E3E70028F8DA06F0E5FE046031
:100400000048FEBDFFFFFF7F1CB50948009009486A
:10041000019005460126009C05E0E36807CC3343C4
:100420000C3C98471034AC42F7D3FFF74DFE000068
:10043000D4870008F48700080048704770720008ED
:10044000F7B582B0029C00272078641C15460197FE
:10045000302802D0002D15D015E020780127641C2B
:10046000782804D0582802D0002D09D00BE0002DA8
:1004700001D0102D07D1002710252078641C02E040
:10048000082500E00A250026009610E000990127C3
:1004900069430818020C294680B2714300908E18F7
:1004A0003804864201D3012001902078641C29463B
:1004B00000F019F80028E9DA0398002805D0002F89
:1004C00001D0641E00E0029C04600198002806D060
:1004D00006F07AFE02210160C81E05B0F0BD009949
:1004E00030040843F9E73A2800D230382023024686
:1004F0009A43412A01D310463738884201D300205D
:10050000C043704780B505F0A5FF002080BD000006
:10051000F8B500241048114E062C16D0075D0025B2
:10052000AF4207D0305D281800F022FA6D1C002879
:10053000F6D002E0641C0848EEE70948009000206D
:1005400008A1424A424B01F0B3FA062C01D3002025
:10055000F8BD0120F8BDC046D6730008DD73000861
:1005600096780008202025732573466C6173685FB8
:100570004572617365506167655F5265636F726450
:1005800073206661696C65640D0A0D0A25730000AD
:10059000F0B5FFB086B01F48016800201E4DA9428B
:1005A00035D0029005A804900C307D218900FFF71A
:1005B00056FE0595042003900090FD20C7000124FD
:1005C000022603253846214632462B4601F076F9AD
:1005D0000690039800900A373846214632462B464B
:1005E00001F06CF90790FFF793FF00F0FDF9049814
:1005F00000F0DCFC002809D008480090002008A189
:10060000124A134B01F054FA204600E002987FB0E2
:1006100006B0F0BD00FE0008A5A4A3A296780008CD
:10062000202025732573466C6173685F5772697467
:10063000655F436F6E666967496E666F20666169C4
:100640006C65640D0A0D0A25730000009B78000894
:100650007C780008F8B5012481256D1E10D00E1D90
:10066000071D096800F016FC0024002831463846B2
:10067000F3D003200349012403A3224606F0CAFC59
:10068000E0B2F8BD847800084253505F466C617355
:10069000685F50726F6772616D5F496E666F50611F
:1006A0006765206661696C6564000000BFB5164827
:1006B00000210A4604F00EFD14490860002805D107
:1006C00003201349012213A306F0A4FC0520039084
:1006D0000A20029015480090032040020190144D1A
:1006E00014A1174A00242846234605F02DF9284670
:1006F00005F0ECF906200649012212A306F08AFC57
:10070000204604B0B0BDC046597800083C0800201F
:100710006378000868725F72785F73656D2063723A
:1007200065617465206661696C656400D0080020AD
:100730004008002068725F746872656164000000A0
:10074000291600084253505F48525F496E69740091
:10075000BFB505F03FFE134DCA2028605320286026
:1007600000F08CF8104805F02DF90120C003FF219E
:10077000EC3100F01DF800F091F800242C60052009
:1007800003210091019002902420082123221423A8
:1007900000F026F80549C81C00F03CF8204604B0DB
:1007A000B0BDC04624280040B80B000080000020E7
:1007B00010B501225303094AD4681C43D46013685E
:1007C000DB03FCD40143D161FF2000043E490A68E9
:1007D00082430A603D480421016010BD0C2800409E
:1007E0001CB51C466B46D8709A70597006981870E4
:1007F000184606F085F8002800D0FEE70599049A0F
:1008000001A881704270047006F0D2F8002800D070
:10081000FEE71CBDFFB50091019007200006029085
:1008200004231449029D144E5B1E21D00F684A68B0
:100830000C684868A742F7D114460F490C40D10212
:10084000294021430392C20230402A400243914290
:10085000039A0849E8D100998F70380A4870380C1B
:10086000087001998A70200A4870100C0870FFBD4A
:10087000FEE7C04600280040FF1FFFFF072040059D
:1008800005490A68824301204305D2180A60C00462
:100890000A6802430A607047182800400948CA21C4
:1008A00001615321016101680422114301600021AB
:1008B0000161FF20000404490B6883430B60034877
:1008C000026070471428004000E400E000E100E00E
:1008D00010B503F0D9FE244CA06840070AD5206863
:1008E000400707D560680421014361601F484068E4
:1008F00004F044FCA06880070AD52068800707D56B
:1009000060680221014361601848406804F036FCC9
:10091000A068000706D52068000703D56068082195
:100920000143616003F0CAFE10BDC04610B503F07C
:10093000ABFE0D48C169890712D5016889060FD53C
:10094000C16902229143C161416820220A43426089
:10095000064CA1682046383003F0A5F80020A060BE
:1009600003F0ACFE10BDC046000002402001002094
:10097000BCB50446104DE868002803D50F48286030
:100980000F4828600F480094019000200EA1144ADF
:10099000144B01F08DF800F051F90220214605F0CA
:1009A000F1FD044600F050F90120C007E968014359
:1009B000E9602046BCBDC04608200240851A7AE5A1
:1009C00091836E7C967800082020257325734572EC
:1009D000617365506167652025640D0A2573000009
:1009E0008E78000878780008E0B57F20FFF7C0FF18
:1009F000002807D004480090002004A14C4A4D4B29
:100A000001F056F88CBDC04696780008202025736A
:100A100025736572726F725F70616765203D202576
:100A200023780D0A0D0A257300000000F0B587B089
:100A30000022026042600490029282602E48425C72
:100A4000039188002D490B5801202D4D0692C4B208
:100A5000944246D805900106CF0B7D190422D11B84
:100A60008126B000C71B761E08D0281D091F3F1F16
:100A7000121F5D596D1C0546F5D104E00598401C18
:100A8000069A1F4DE3E7D81B069DAC420DD2591ABA
:100A90000A68521C1DD0049A5160906054800398DB
:100AA00040001849085A108023E0991A049A5160AE
:100AB00090605480039840001249085A1080012C1D
:100AC00017D11146536093601868401C11D10298E9
:100AD00005E004994B6088604C807842800808806B
:100AE00007E009480090002008A1D64AD64B00F044
:100AF000DFFF07B0F0BDC046D6730008E4730008FE
:100B000000FEFFFFC87300089678000820202573B8
:100B10002573466C6173685F476574496E646578D8
:100B20005F506F73204572726F72210D0A2573003A
:100B30009B7800087C7800081FB5014601AC204670
:100B4000FFF774FF207804B010BD0000F0B58BB043
:100B5000471E062F34D814460D46F9B20AAE304669
:100B60002A4600F079F87178B37832781609099638
:100B70000396009701951D06AD0E089506951B027C
:100B800059181F270F4004970F261640002802D13E
:100B9000FD20C000361802968805C50E0595072071
:100BA0000949012209A306F035FA089860712571F8
:100BB000E7700998A0706670300A2070002000E08D
:100BC00001200BB0F0BDC0468478000828256429B8
:100BD000466C6173685F4765745265636F72645BEE
:100BE00025645D3A253034642D253032642D25305E
:100BF00032642C253032643A253032640000000023
:100C000070B5044600250C4E2846B04720800120D0
:100C1000B04760800220B04720710320B047607168
:100C20000420B047A0710520B047E0710620B0470E
:100C30002072284670BDC046390B000880B5FFF70A
:100C400059FA0449086080BD80B502480068FFF782
:100C500055FA80BD700F0020F0B591B016460D46D4
:100C600004460EA8FFF7E2FE68006349085A711EA9
:100C700081420AD20EA80288B24219D26048009678
:100C8000019202900025824905E05D49009601909D
:100C9000029100255BA16B4A6B4B284600F008FFD0
:100CA000E570A570657025700125284611B0F0BD6E
:100CB000A80052490858B1000F9F87420D920B9728
:100CC00002D10818001F21E04A4A525D7B185202E7
:100CD0001018091F0C9183420DD9494800970190C3
:100CE000002066490A92634A634B00F0E1FE0C98CB
:100CF0000A99401A09E0424800970190002053A148
:100D00005C4A5D4B00F0D4FE0C98C0190C9007684B
:100D1000384601F01FF8390E884240D12770E17043
:100D2000380CA0703A0A62703802800E0A90B9033B
:100D3000C90E1F2313403A06120F0F203840FD271B
:100D4000FF00C0190095019602AD0DC505910A98E6
:100D500006902B4E079600254B49464A464F28469B
:100D60003B4600F0A5FEE078A178227863780EACCF
:100D700064881B029A1809040006401880180B9911
:100D800000910C9901910D9902910394049005969C
:100D90003E492846374A3B4600F08AFE85E70A91DD
:100DA0000EA94A88164B09900B9900910C98019056
:100DB0000D9802A985C1059300263149214F224B88
:100DC00030463A4600F074FE0D980090019509985F
:100DD00002900A9803900C980490094805902949BC
:100DE00030463A46184B00F063FEE670A670667017
:100DF000267059E7D6730008C8730008E47300082A
:100E000096780008202025732573696E6465782024
:100E10006E756D2028256429203E20687220726539
:100E2000636F7264206D6178206E756D202564207B
:100E3000262620696E646578203E20300D0A2573D1
:100E4000000000009B7800087C78000820202573B3
:100E5000257372656164203A68725F73746172749D
:100E60005F6164647231203D202523780D0A25736B
:100E7000000000008E78000878780008587D00088F
:100E80003F7A00080C790008E17C0008AB78000884
:100E90006D7C0008F0B585B0044680070AD0009448
:100EA00003202349012523A32A4606F0B3F8284648
:100EB00005B0F0BD0E46264F1C20B860F86800282B
:100EC00003D52448386024483860F8680025002895
:100ED000EDD40495FFF7B2FE2046314605F098FBAD
:100EE0000546FFF7B1FE002D0ED02068009401905A
:100EF00007200F49012519A32A4606F08BF8E807B9
:100F0000F9680143F960D2E70125E807F968014370
:100F1000F9602068B04204D1022004F053FD049D22
:100F2000C5E70094019602900720014910A3BBE792
:100F30008478000861646472202523582069732036
:100F40006E6F7420616C69676E65640D0A00000045
:100F500008200240851A7AE591836E7C6164647290
:100F6000203D202523582C207265616420256400D3
:100F7000466C6173685F577269746520446174617F
:100F8000204D69736D6174636820617420616464CD
:100F900072202523582C2065787065637465642061
:100FA000256420676F7420256400000080B5014629
:100FB0000148FFF74FFB80BD00FE0008F0B597B079
:100FC0000446062816D179480068411C12D01690B4
:100FD0007748012700240625009501940297039085
:100FE0007449754A754B204600F062FD16A82946E3
:100FF0002246D5E013A812902146FFF717FD16AE42
:1010000000201090F0706E490A7813090A204343BB
:10101000D21808320F231A401F464B7811941D092D
:101020004543EB181B019A183270664B1A78150964
:101030003C463A404543AD181F220F9215400E958D
:101040006D015B781F09234022460B944743FB1830
:101050003F241C400D94A3025B191C0A0994B47030
:1010600089780F091140474378180F9908400C9070
:101070001C1874701298078840881290149D159857
:101080000890169800F066FE0A900999B1701199BF
:101090007470F070169E464809950095089C01945E
:1010A0000F970297129A03920D46049605904649AF
:1010B000464A474B109F384600F0FAFC3006000FB6
:1010C0000B9A3240FD21C900511800950191029000
:1010D0000C9803900E9804900D9805900A9806902D
:1010E000334807903B493846384A394B00F0E0FC1A
:1010F000254620463146FFF7CDFE00281BD02C4860
:101100000090002434A12C4F2C4B20463A4600F08E
:10111000CFFC0998009001950F98029012980390C7
:10112000049623480590344920463A46234B00F064
:10113000BFFC012736E00F9E119880002F49085808
:10114000129949020818001F85421FD100951848BE
:10115000019000202A492B4A2B4B00F0A9FC2B4878
:101160001199445C2A48405C1299814201D212983C
:1011700024182046FFF7FCFB002807D000940C48F9
:101180000190002023491F4A1F4BD0E711984000CF
:101190002149085A3246864200D2521C16A811999B
:1011A000FFF75AFD384617B0F0BDC04600FC0008F6
:1011B00096780008FE7900089B7800087C78000883
:1011C0008300002080000020DF7A00088E7800086D
:1011D00078780008977B00082020257325736872B3
:1011E0005F77726974655F646174615F6572726F65
:1011F000720D0A25730000003E7B0008E4730008AE
:10120000E27B0008A378000880780008DD730008FE
:10121000D6730008557C0008C87300080022002916
:1012200004D003789A18401C491EF8E7D0B27047E2
:10123000FEB50293009201910446089FB81D2070EC
:10124000661C0120020200253046294603F0A6FB59
:1012500027710098E0700198A070AA206070601D4E
:1012600002993A4603F082FB2078871E30463946C1
:10127000FFF7D4FFF05520788019401E55210170EA
:101280002846FEBDF8B5074600250091A94214D0B6
:10129000785DAA280FD17E19F47830194079552845
:1012A00009D1211D3046FFF7B9FF391949190979CC
:1012B000814200990AD06D1CE8E7032012490122FF
:1012C0001EA305F0A7FE00252846F8BDE01C03F08C
:1012D00059FA002813D0054670782870B078AC70A1
:1012E0006870002C04D0311DE81C224603F03EFB40
:1012F00007200549012205A305F08CFEE4E7032041
:101300000149012208A3DCE76378000848525F47DF
:101310006574446174614672616D652053756363E1
:10132000657373210000000067657420737061634A
:1013300065206661696C0D0A0000000048525F4735
:101340006574446174614672616D65204661696CC3
:1013500021000000F0B5DFB005460EA84021FEF7E1
:101360007EFF6C782D78082C22D8A00001A10858A7
:101370008746C04699130008B5130008E11300081A
:10138000F5130008091400081D14000831140008A2
:101390007F140008B114000807268B490122A14BD5
:1013A000304605F037FE0EA8FFF72AFC00254CE07A
:1013B00000264AE00095072683490127984B3046CE
:1013C0003A4605F027FE0EA938460F4629463A460A
:1013D000FFF7BCFB002838D03878002861D034E013
:1013E00000950726784901228C4B304605F012FE05
:1013F000022026E00095072673490122864B3046DD
:1014000005F008FE03201CE0009507266E49012226
:10141000804B304605F0FEFD042012E000950726C3
:101420006949012275A3304605F0F4FD052008E066
:1014300000950726644901226BA3304605F0EAFDBA
:1014400006200EAA2946FFF781FB601EC0B20528C0
:1014500006D8002D04D10EA80021324603F09EFAD2
:1014600000961EAE0EAB304629462246FFF7E0FE40
:101470003178701C00F0A8F900205FB0F0BD009535
:1014800007265149012751A330463A4605F0C2FDCF
:101490000EAA30463946FFF759FB0028D5D0002D5B
:1014A0005ED00EA800210726324603F077FACCE77B
:1014B0001EAF00200B90B87038800DAE0C96B07047
:1014C000308030463946FFF7A5F971780F220B09B5
:1014D00011400A26734358180A900EA988700C9878
:1014E0008378180913407043C0180990C870387881
:1014F000030910407343181808900871787803099D
:10150000104073431B184B71B8780709104077439C
:10151000381888710C9F3F783A403F097743BA18D2
:10152000D6B2303A4A707D221201B218160A0E70F5
:10153000C1B2DBB20898C6B20998C7B20A98C0B265
:101540000092019002970396049305910AA00690D9
:101550000BA11AA21BA30B9800F0AAFA072674E7A6
:101560000EA84078002802D00EA807701EE70EA82B
:1015700000250726294697E71B5B306D0000000019
:101580002020257325736B47657443757272656EF1
:101590007454696D653A20253034642D25303264E9
:1015A0002D253032642020253032643A25303264D3
:1015B0003A253032640D0A25730000001B5B313B75
:1015C00033326D00493A2000637800086B53656E32
:1015D000736F724661696C7572655265636F726490
:1015E00028256429000000006B506F7765724F6EEC
:1015F0005265636F72642825642900006B506F7711
:1016000065724661696C7572655265636F726428B4
:101610002564290045780008207800083178000802
:101620000F7800086A7800088AB002A82021FEF727
:1016300016FE204C214D204E20680021C94303F0A6
:10164000E1FD072401220192204631462B4605F098
:10165000E1FC1B4D284602F0AAF9C7B200972046CC
:101660003146019A17A305F0D5FC02AC2846134D6C
:1016700021463A4602F0BEF9102116A022460D4C32
:101680003B4605F0A7FB062FD6D302A83946FFF745
:10169000F9FD0746002808D0BB78FA1C102111A0DC
:1016A00005F098FB3846FFF755FE384602F036FE47
:1016B000C2E7C0463C08002063780008597800085B
:1016C0006C0100206275665F6C656E203D202564AC
:1016D0000A0000006C7075617274315F72785F721D
:1016E00062000000486F73744672616D65446174F6
:1016F000610000007CB502F0C7FF01A80021017065
:101700003D4E306880060AD5F069800607D5706ABC
:1017100001A908705C484C30012202F0E8F93068F9
:10172000000616D5F069000613D5574C60342046E4
:1017300002F03DF9002808D001AD012220462946DB
:1017400002F058F92878B06203E0306880218843BD
:1017500030603068400607D5F069400604D5402067
:1017600030623168814331603068C00707D0F0696A
:10177000000704D540203062706A01A9087002F0A9
:101780009DFF7CBD70B50C4605463F4E30464C3043
:1017900031461431102202F01EF9603608498022C9
:1017A000304602F018F900F029F82846214600F0EA
:1017B00023FD062035490122024B05F02BFC70BDAC
:1017C000740F0020A285000870B50C4605462E4E09
:1017D0006036304602F0D6F8A04201D2002070BD3B
:1017E00030462946224602F082F903490A688023DE
:1017F00013430B6070BDC04600800040F0B587B059
:101800001148016802263143016000BF00BF00BFDC
:1018100000200190059003960127F802029006240B
:1018200006940497094802AD294604F009FF01987F
:1018300005900396B802029006940497034829463F
:1018400004F0FEFE07B0F0BD2C1002400004005072
:10185000BCB50D4D28464C3002F0A9F804460028CE
:101860000ED02868A0420BD100940720074901221E
:1018700007A305F0CFFB0B48006803F07FFC01E0F5
:10188000002C00D02C60BCBD20010020AE850008DB
:101890006C7075617274315F72785F72623A202584
:1018A000640000003C0800200120000202490A6890
:1018B00002430A607047C0461810024010B5083055
:1018C0000F24044008012018C0B21F211140DA067D
:1018D000920D5118029A9206120C891809020C18DE
:1018E000204600F037FA0006201810BD80B502F03F
:1018F000CBFE15484168890404D5016C890701D5E0
:101900000221816411490A68D20704D08A68D2078B
:1019100001D001220A614168C90404D5016CC907DC
:1019200001D0012181640168490709D5016C49038F
:1019300006D50121890481640549C81CFEF76AFFA8
:1019400002F0BCFE80BDC046142800402CB0004010
:1019500080000020BCB5002401AD012220462946AC
:1019600000F00AF8012801D0E043BCBD2878BCBDD6
:1019700080B500F005FC80BD10B50B46EFF3108478
:10198000012181F31088194600F004F884F31088CF
:1019900010BD0000FEB50B460546444C2078532888
:1019A00005D01E46174600F0EBFB3A46334618209A
:1019B00068432418E76E266FBE4217D9606E029204
:1019C000A26E8119951B0298854200D305460193AA
:1019D00018462A46FEF72AFC029AAE19A06E8642E5
:1019E00000D10026521B019B5B1900E00025BF1BA4
:1019F000974200D31746002F07D0606E8119184612
:101A00003A46FEF713FCBE197D19002D01D0703443
:101A100026602846FEBDC046F8B514460D4606466B
:101A200022480078532801D000F0AAFBEFF310877A
:101A3000012181F3108830462946224600F004F83F
:101A400087F31088F8BDC046F8B514460D46182136
:101A5000414316484618F06A1836022810D001286B
:101A600015D0002700281ED1304600F0B9FBA04257
:101A700019D330462946224600F0A2FD274612E03F
:101A800030462946224600F06DFD07460BE0304601
:101A900000F0A6FB0746A04200D327463046294661
:101AA0003A4600F08DFD3846F8BDC046D001002012
:101AB00082B0E0B50492059304AA019201AA00F055
:101AC00005F88CBC02BC02B008470000F0B59FB01E
:101AD00007920E4602901E9000271C9740201B90F4
:101AE0000AA81A901D9731783046761C252906D011
:101AF000002900D11AE11AA800F03EFC90E0801CF9
:101B000000253178232907D02B2907D02D2907D08C
:101B100030290AD1022104E0082102E0042100E07A
:101B200001210D43401C761CEBE700240897302967
:101B300009D3392917D80A2262435418303C401C73
:101B40007178761CF3E72E290DD100270921CA43AD
:101B500001780B463A3B934207D30A227A4357183F
:101B6000303F401CF2E7002700E00646761C08469E
:101B7000633809280DD8C04678440079400087446E
:101B8000545A4F4F4F044F4F4F04701C3178064644
:101B9000EDE708467038082815D8C0467844007923
:101BA00040008744043D3D1E3D313D3D1400079AF1
:101BB0001068011D11600168002008230093019046
:101BC0001AA810222AE0252958D0582928D1079A86
:101BD0001068011D11600168009401951AA8102277
:101BE0001BE0079A1068011D11600468002C00D1E9
:101BF00056A42178002913D01AA800F0BDFB641C5C
:101C00001D980028F5D50BE0079A1068011D11609A
:101C10000168009401951AA80A223B4600F02AFBAD
:101C20001D9F002F00D45EE78DE0079A1068011D0C
:101C3000116001785FE7079A1068011D1160026862
:101C4000D01711464140081A0692514204910121D1
:101C500009910A2805D30A21FEF75EFB0999491C60
:101C6000F6E70998B84200D80997002C09D00698E1
:101C7000002801D4680705D5641E03E01AA82521B1
:101C80003AE70024022129400596039101D0002F54
:101C900013D0E80711D1002C0FD0661EA6420CD23B
:101CA0000998A04209D21AA8202100F065FB1D98CE
:101CB000089000283446F0D521E008980028059EB9
:101CC000AED40698002804D4680704D4069804907B
:101CD0000AE02D2102E02B21069804901AA800F0BA
:101CE0004BFB1D9800289BD40398002809D1009431
:101CF00001951AA80A2204993B4600F0BBFA059EFA
:101D00008EE7012028403843F1D1002CEFD0661E29
:101D1000A642ECD20998A042E9D21AA8302100F0DC
:101D20002BFB1D9800283446F1D5E8E7002F09D099
:101D30001C9D002D04D00AA902982A46FFF76CFECC
:101D4000EF1900E0002738461FB0F0BD284E554C73
:101D50004C2900000F2101400206120F5118C20445
:101D6000D20E89188203D20E89180002800E08183C
:101D7000704780B502F088FC03F0CAFF02F09EFCB9
:101D800080BD000010B51D4CA0688006400F411EAC
:101D9000032922D81A48C0467944097949008F445A
:101DA00021011619E168C90700D11E48E16809063A
:101DB000C90E00D120214843E1684905490F00D1EF
:101DC0000821FEF7A9FAE1684903890F09E07D209F
:101DD000000207E00120C00304E02068C004810F76
:101DE0001048C840A16889091C220A400549895841
:101DF000FEF792FA0A49086010BDC0460010024082
:101E000000127A00A87300080348044901600448DE
:101E1000044901607047C04608ED00E0000000087A
:101E20000C0000200024F40000F0E6FBBCB50C46DA
:101E30000021019103280CD16068FEF74BFA05469A
:101E4000A068FEF747FA0246E9B201A8FEF704FFD0
:101E5000BCBD03200249012202A305F0DBF8BCBD92
:101E600084780008544553545F466C6173685F5230
:101E70006561645F5265636F7264202020202020BA
:101E80002D2D757365205F636D645F205B726563E4
:101E90006F726428307E36295D205B6E756D5D0043
:101EA000FEB503281FD10C464868FEF713FA054615
:101EB000A068FEF70FFA0446EDB201262A4FA642AB
:101EC00017DC009501961C48029000201BA1244AB3
:101ED000244BFFF7EDFD2846FFF770F8384603F076
:101EE00071FD761CEBE703200249012202A305F0F5
:101EF00091F8FEBD84780008544553545F466C61E8
:101F000073685F57726974655F5265636F726420AE
:101F100020202020202D2D757365205F636D645F68
:101F2000205B7265636F726428307E36295D205BAA
:101F30006E756D5D00000000967800082020257306
:101F40002573466C6173685F57726974655F2825F5
:101F500064295265636F72643A25640D0A25730023
:101F6000A37800088078000860EA0000F8B50C4605
:101F70000546804F384624300C49802201F02BFD65
:101F80003837012672020A49384601F024FD00F074
:101F900039F800F093F82846214600F0A1FA06200F
:101FA0006D49044B324605F035F8F8BD2813002082
:101FB000201C0020A285000880B502F065FB1048B7
:101FC0000168C90504D5C169C90701D001210162B1
:101FD0000168C90704D0C169C90701D001210162A4
:101FE0000168C90608D5C169C90605D51021016275
:101FF000F548406803F0C2F802F060FB80BDC046BF
:1020000000380140F0B587B0224801680125294316
:10201000016000BF00BF00BF0627029700260096A0
:10202000E8020690059610200490039601966C46EF
:10203000204604F075FA02970095069605960496D8
:10204000202003900196204604F06AFA124C206882
:10205000022101432160206804210143216020689E
:10206000082101432160FF2001020C4A13688B43C1
:10207000136069027E4B196000041168814311608E
:10208000A80218603D4800F00BF820682843206043
:1020900007B0F0BD301002400800024008E400E044
:1020A000F8B5802103910290034801900020009030
:1020B000684604F053FA8FBD24380140F0B587B06C
:1020C0001248016801263143016000BF00BF00BF14
:1020D00000200190059002270397F00202900696D7
:1020E00004960520040702AD2046294604F0A8FA0C
:1020F00001980590039730030290069604962046B7
:10210000294604F09DFA07B0F0BDC0462C100240ED
:1021100007201149012211A304F07CFFD04E164F75
:1021200070680021C94303F06DF83C6880210D1BE5
:1021300032699542F4D011488018954201D9A91A04
:1021400006E0891A00F038F9802C03D00B482946A4
:1021500000F032F93561E3E7AE850008556172742D
:10216000315F52785F5468726561645F456E747266
:1021700079000000200100200C00024088060020A9
:1021800010B5124CA8212046FEF769F80320206103
:1021900060610F49A1610F48E06101208002206267
:1021A0000020A0626062E06221660B496166102136
:1021B000A1662067E066606708490F31102804D0E7
:1021C0000A782254491E401CF8E710BDD0010020B7
:1021D000B785000888020020780200207472000889
:1021E000C2680169914201D9D04302E0D243891803
:1021F000806808187047000070B588B00022079208
:1022000003239B02174CA6689E430125EB02F3189B
:10221000A3602B0526681E43266000BF00BF00BFD9
:10222000069103900192059204920C2002900E4CAC
:1022300001A9204604F051FA002800D0FEE70B481F
:10224000016840220A43BF218A4302602807C4492B
:102250000860206820210143216020682843206015
:1022600008B070BD34100240008000401CE400E063
:1022700000E100E0F0B587B0039317460590012612
:102280000D9D0C9C01910846B84204D33946FEF7D7
:1022900043F8761CF8E706970127039B9E4200D877
:1022A0001E4628463840002C0496029018D000287C
:1022B00016D12020A90701D4054600E03025002BC7
:1022C00000D00546002C0BD0A64209D2059E304610
:1022D000294600F051F8641EF068049E0028F1D5EC
:1022E0000598C06800283DD40094019D039C022CF1
:1022F00002D3641E069906E028463946FEF70CF81C
:102300000699884201D34F43F1E7059E2846394696
:10231000FEF702F8044614A0015D304600F02CF8E8
:10232000F068002809D47C432D1B3846069C2146C2
:10233000FDF7F2FFA7420746E8D202980028049E64
:1023400000980FD000280DD0059D441E844209D26C
:10235000864207D22021284600F00EF8E8680028BF
:102360002046F2D507B0F0BD303132333435363740
:10237000383941424344454610B5044642688368B3
:10238000581C904201D9184606E02268D154A0603A
:10239000E168491CE1606268904208D121682069C7
:1023A000FFF73AFBA168884202D10020A06010BD6F
:1023B0000020C043E06010BD80B50A4601462848B1
:1023C000243001F094FB80BD200100201FB51FA028
:1023D0000021012202F07EFE214C6060002807D11E
:1023E00020480090002020A12BA22DA3FFF760FB26
:1023F000022000902BA02E4900220A2303F034FD76
:10240000E060002801D003F0C3FD052003901420F4
:10241000029028480090FD20C0000190264827A186
:102420002A4A002303F090FA00280BD1224803F037
:102430004DFB0C49009001910020254925A227A3BE
:10244000FFF736FB002004B010BDC0467561727402
:10245000315F72785F636865636B5F73656D000001
:1024600020010020967800082020257325736372D0
:10247000656174652075617274315F72785F63683D
:1024800065636B5F73656D2063726561746520665B
:1024900061696C0D0A2573001B5B313B33306D00A5
:1024A000443A20006C7072785F74696D65000000BA
:1024B0005118000838140020A813002075617274A8
:1024C000315F72785F746872656164001121000881
:1024D000708500081B5B313B33326D00493A2000A8
:1024E000B0B588B00125AA031A4B1C6814431C60C0
:1024F00000BF00BF00BF0022079206910592049220
:1025000003900C2001900292134C01A9204604F084
:102510009FFA002800D0FEE7FF2000020F490A685A
:1025200082430A6068060E49086028022168014358
:102530002160206828432060206810210143216029
:10254000A06840210143A16020682843206008B0B2
:10255000B0BDC046381002400038014018E400E029
:1025600000E100E0FEB516460D46C7680021019067
:102570000269BA42029103D9F9435418816803E011
:10258000F9435218816854184268C91B8C4200D321
:102590000C46B44200D33446D01929462246FDF7F2
:1025A00045FEE719019881688F4200D10027029902
:1025B000C760361B2D196118002ED9D10846FEBD03
:1025C000F8B5154604464068A268E6688019971B6E
:1025D000BD4204D22A46FDF729FE751909E00E46D0
:1025E0003A46FDF723FEF119ED1B60682A46FDF718
:1025F0001DFEE560F8BD0000BFF34F8F034804499E
:102600000160BFF34F8F00BFFDE7C0460CED00E057
:102610000400FA0580B5012000F086FC80BD7047FB
:10262000002804D0C1B2002903D0012010E000200E
:102630007047FF210A02024002D0110A092007E078
:102640000904014002D0090C112001E0010E1920FB
:10265000014A515C4018704785720008FEB50120A0
:1026600000F062FC0B4F009700240BA1124D134E9B
:1026700020462A463346FFF71BFA114800680090AF
:10268000019710A120462A463346FFF711FA20464B
:10269000FEBDC046967800082020257325735F7024
:1026A0006572665F636F756E7465725F696E69747B
:1026B0000D0A257300000000A37800088078000848
:1026C0000C000020202025732573706572665F63FF
:1026D0006F756E74657220696E69742C20537973FE
:1026E00074656D436F7265436C6F636B3A25640D5F
:1026F0000A257300FEB50446089D064628362EC6F8
:102700001C30E0612062232118462A4602F046F977
:10271000234628330FCBD218121F144B01F080FF31
:10272000606225463C350A9E099F202F04D310A0E5
:1027300018A1A72201F06EFD6F70AF70E6642665E8
:1027400000202064A063E864286528700090019050
:1027500020465430134A2146234603F0EDFB12482D
:102760000168002901D020468847FEBDFD570008BA
:102770007072696F72697479203C2052545F5448BA
:10278000524541445F5052494F524954595F4D415F
:10279000580000005F72745F7468726561645F69FD
:1027A0006E697400F55B00081411002070B50546D1
:1027B0008826FDF79FFC0446A959002901D0284628
:1027C00088472046FDF79AFC70BD00000B4A02289E
:1027D00006D0012809D1032003051068984302E0C0
:1027E00001204104106808431060012000041168B2
:1027F0000143116010684003FCD57047001002408F
:10280000074908684A68801A064A1268520106D5C4
:102810000A68121A102A02DB09684018401C704727
:1028200014E000E004ED00E080B500F05BFD002066
:1028300080BD80B500F044FF002080BDF0B58BB0B6
:102840001E460A920D460746109C01F02DFF0028F7
:1028500009D000960194002039462A460A9B04F0CC
:10286000D3F90BB0F0BD09960795354801680029EA
:102870000A9AF6D0456B002D5ED02346B800314948
:1028800008180590A620F840012101400691201F5C
:1028900003900894002DE4D0284618380068B84208
:1028A00048D32E462C3E281F0468002C0BD00998D4
:1028B0000090019330463946079A0A9BA047089B2F
:1028C0000A9A002836D028461C38006810430DD0DC
:1028D000284610380468099800900193304639461C
:1028E000079A0A9BA047089B0A9A23E006980028AB
:1028F0001846099C214611D10598006802F071FD27
:10290000024600280898214608D00F48049202F099
:1029100068FD049941180398401A61182A46103A34
:10292000146800910190002330463946079AA04769
:102930000A9A089B2D68ADE7099801F013FF90E70C
:10294000201E002088730008E785000810B5154890
:1029500041692922895C890703D413480021017049
:102960001EE00169002905D0012002020E48FDF792
:1029700081FC15E001F09CFA002803D00A480BA165
:10298000052202E008480BA10722FDF74FFC064C88
:102990002046FDF77CFC3E21215420180021417087
:1029A000014810BD88000020380700206D736820A2
:1029B0000000000066696E7368200000B0B5044630
:1029C000094D6869002805D1084809A1A42201F031
:1029D00021FC68692921425CFD231340E207920F24
:1029E0009A184254B0BDC04688000020047E0008FA
:1029F00066696E73685F7365745F70726F6D707413
:102A00005F6D6F6465000000FEB5184F18481949E6
:102A100039607860852081000125284601F030FC6E
:102A2000786100281AD00A20152100910190AB028C
:102A300011A013490024224602F0EAFD06467869F7
:102A400010A12246234602F075FB2846FFF7B6FF89
:102A5000002E08D0304603F039F804E00BA001F056
:102A60006BFE0020C4432046FEBDC0468800002007
:102A7000D48700089C860008747368656C6C00003D
:102A8000A52A000873687278000000006E6F206D40
:102A9000656D6F727920666F72207368656C6C0A61
:102AA0000000000084B0F34D68692922815C012395
:102AB0000393194302928154FFF748FFEE4801F057
:102AC0003BFE01F029FD07466C69204628301B2F8C
:102AD00002D103990170F4E7E849661801780229E8
:102AE00006D0012935D15B2F31D102210170E8E7F1
:102AF0000021017038460838052871D93846413818
:102B0000032832D84000C04678448088400087447B
:102B100003006D0174018701608D002800D1A6E1DA
:102B2000401E6085DF214900651880B25022504365
:102B300021182E312846FDF779FB2846CD4DFDF7AB
:102B4000A6FB70803080204603F09AFCB9E7002194
:102B5000017038460838052807D8C04678440079FF
:102B6000400087446A9E45080845002FA9D07F2F62
:102B700063D0FF2FA5D03088502801D300203080AB
:102B80007188814200D3E4E0421A6118FF20C0300E
:102B90000818DF232E465D00491901F0E7FE2120C9
:102BA00004017069015B4018475570690299415CE6
:102BB000C90707D00119098840184119B7A001F0C9
:102BC000BBFD70693546045BAE4EAC49415A8C4240
:102BD00000D3CCE0304601F0AFFD641C6869F4E737
:102BE0007844007940008744285C03020203C2E76E
:102BF000A58D3088002800D1D5E0052D7ED3B720E3
:102C000040002718DF20400021185022384601914B
:102C1000FDF744FB002800D1C5E0009725467E352E
:102C20000427002F00D1B2E0284650385022294610
:102C3000FDF7FCFA7F1E5035F3E77188002900D1BB
:102C40003FE7481E70803288521E328080B292B2B6
:102C5000824272D9121ADF235D00631918185918BD
:102C600001F084FE834840698449415A401800219C
:102C70004155212004017F484069015B40184119FA
:102C80007C4D83A001F058FD6869045B7B49405A84
:102C9000844200D915E77B4801F04EFD641C686949
:102CA000F4E70025774E21200001205A854206D204
:102CB000304601F041FD6D1C6E484469F3E77248EF
:102CC00001F03AFDDF204500641901F0F1F8012818
:102CD00002D1204600F070FFFFF738FE6E486649CB
:102CE000224601F029FD63494C6960190D46FDF744
:102CF000CEFA6249605261184880E2E6002D0BD09E
:102D0000DF20400021185022104668430019223865
:102D1000FDF7C4FA002846D050214D4365192E35E1
:102D20002846FDF79CFADF2040002118328828460B
:102D3000FDF77CFAA08D451C34E054A001F0FCFCAA
:102D400068694E49415A4018DF2149000022425427
:102D5000B7E62018DF214900475468690299415CB1
:102D6000C90704D04648394601F0E6FC6869434A81
:102D7000815A491C815280184288521C428089B273
:102D8000502900D29DE600214180018099E6502122
:102D9000009D2846FDF763FA328828460199FDF721
:102DA00045FA0525A585658501F082F80128314D94
:102DB0000FD168690299415CC90703D0324801F01C
:102DC000BBFC68692D49415ADF225200801800F08F
:102DD0004BFFFFF7BBFD284801F0AEFCDF204000B1
:102DE000696908185421FDF73AFA6AE6618DA28DE7
:102DF000501E884222DD481C23E0708831888842BA
:102E000000D35EE62018DF214900415C1C4801F038
:102E100093FC2120000169690A5A521C0A5250E6AB
:102E20007088002800D14CE6164801F085FC21206E
:102E3000000169690A5A521E0A5242E6002A00D16C
:102E40003FE66085DF214900651880B2502250437B
:102E500021182E312846FDF7E9F92846FDF717FA23
:102E600070803080204603F00BFB024D29E661851F
:102E700027E6C04688000020380700200E02000028
:102E8000157E0008027E00088F7E000808200800DA
:102E90000825732020080000187E00082573000014
:102EA00010B5064C01F000FC002803D0052080017D
:102EB000241800E03834204610BDC046201E0020F3
:102EC00070B5EFF31084EFF3108072B600252A4E30
:102ED00028462946002D15D1FFF792FCC217716ACA
:102EE000336A18185141F26AB36AC31A0B46934108
:102EF00002DAF16AB06A01E0B062F16284F310882C
:102F00002D1FE7E770BDC04680B502A001F014FC9C
:102F1000002080BD48656C6C6F2052542D5468723F
:102F2000656164210A00000070B5EFF31081EFF3D2
:102F3000108272B600220F4B114C104D002A0ED198
:102F4000002805D100261E605D609E6007261E6079
:102F500001267606266081F31088121FEEE704F042
:102F600003F9054800214162016281600161FFF7B8
:102F700056FB70BD10E000E0A0010020FFFFFF0045
:102F800004ED00E0F8B50EA001F0D6FB114805688D
:102F90001148076811A4AF4210D23E6802223046A1
:102FA0002146FDF788F9002806D07A680CA0314642
:102FB00001F0C2FB074805680C37ECE70020F8BDBC
:102FC0002D2D46756E6374696F6E204C6973743A6B
:102FD0000A0000008C000020880000205F5F0000D5
:102FE000252D313673202D2D2025730A0000000079
:102FF000F0B595B00424204601F030FF10A90C7202
:10300000002414940821139108A91191001D109017
:1030100028A0102130A201F08FFB00F04BFF30A060
:1030200001F08AFB0394204610AC214600F080F8A2
:103030000490207A069008AE14980790039D079894
:10304000854230DA3468271FFDF754F83F78FDF7E2
:1030500055F87F2038400699884221D12746143FF1
:103060002169A0680834A04213D02046059101F0E0
:103070007FFB059900910190102121A00A463B4653
:1030800001F05AFB204603F013FA234801F054FBE9
:1030900006E00091102121A00A463B4601F04CFBBE
:1030A000361D6D1CCBE704980028BDD1002015B05B
:1030B000F0BDC046252D2A2E73202020202020730D
:1030C00065742020202073757370656E64207468A9
:1030D000726561640A0000006576656E7400000028
:1030E00020202D2D2D2D2D2D2D2D2D2D202D2D2D37
:1030F0002D2D2D2D2D2D2D2D2D2D2D0A00000000D7
:10310000252D2A2E2A732020307825303878202546
:103110003033643A000000008F7E0008252D2A2EEF
:103120002A73202030782530387820300A000000BB
:10313000F8B5064600250D61C868002828D00C4661
:10314000087A002824D000952768002E3D4600D03C
:103150003546FCF7CFFF002E06D0311F09787F22BD
:103160000A40217A8A4210D1626800210E462D68F9
:10317000BD4205D020C2761CE3689E42F7D100E034
:103180000D46FCF7BBFF266102E0FCF7B7FF009D90
:103190002846F8BDF0B597B00524204601F05EFE44
:1031A00012A90C7200241694082115910AA91391F2
:1031B000001D12902CA0102134A201F0BDFA00F0E5
:1031C00079FE34A001F0B8FA0394204612AC2146EF
:1031D000FFF7AEFF0490267A0AAD1698089003997F
:1031E00005960898814239DA09912C68271FFCF767
:1031F00081FF3F78FCF782FF7F203840B04229D121
:1032000007952746143FA58AE08A0690A6680834E9
:10321000204601F0ADFAA64210D006990091019522
:103220000290102122A00A463B4601F085FA204672
:1032300003F03EF9244801F07FFA09E00699009175
:1032400001950290102121A00A463B4601F074FA34
:10325000059E079D2D1D0999491CC2E70498002869
:10326000B4D1002017B0F0BD252D2A2E7320656E35
:103270007472792073697A652073757370656E64F2
:10328000207468726561640A000000006D61696CF9
:10329000626F7800202D2D2D2D20202D2D2D2D20FD
:1032A0002D2D2D2D2D2D2D2D2D2D2D2D2D2D0A009E
:1032B000252D2A2E2A7320253034642020253034F1
:1032C000642025643A0000008F7E0008252D2A2EF8
:1032D0002A7320253034642020253034642025646E
:1032E0000A000000B0B5064DA96806A00A4CA04728
:1032F000A9690AA0A047E9690DA0A047B0BDC046D2
:10330000AC000020746F74616C206D656D6F727914
:103310003A2025640A000000394700087573656487
:10332000206D656D6F7279203A2025640A000000D7
:103330006D6178696D756D20616C6C6F636174652A
:1033400064206D656D6F72793A2025640A00000073
:10335000F0B595B00624204601F080FD10A90C724E
:10336000002414940821139108A91191001D1090B4
:1033700029A010212FA201F0DFF900F09BFD30A061
:1033800001F0DAF90294204610AC2146FFF7D0FE96
:103390000390267A08AD1498069002990496069830
:1033A000814233DA07912C68271FFCF7A3FE3F7890
:1033B000FCF7A4FE7F203840B04223D10595274674
:1033C000143F258BA6680834204601F0D1F9A642A7
:1033D0000ED00095019010211FA00A463B4601F037
:1033E000ABF9204603F064F8204801F0A5F907E0A6
:1033F0000095019010211EA00A463B4601F09CF961
:10340000049E059D2D1D0799491CC8E703980028B7
:10341000BAD1002015B0F0BD252D2A2E7320656E7F
:103420007472792073757370656E64207468726548
:1034300061640A006D736771756575650000000051
:10344000202D2D2D2D20202D2D2D2D2D2D2D2D2DD3
:103450002D2D2D2D2D0A0000252D2A2E2A732025F5
:10346000303464202025643A000000008F7E00087C
:10347000252D2A2E2A732025303464202025640A25
:1034800000000000F0B597B00324204601F0E6FCF0
:1034900012A90C7200241694082115910AA91391FF
:1034A000001D129022A010212AA2069101F044F9D9
:1034B00000F000FD29A001F03FF90494204612AF6E
:1034C0003946FFF735FE0590387A08900AAD169810
:1034D0000990049E0998864224DA2F683C1FFCF765
:1034E00009FE21787F220A4008998A4215D1FCF70B
:1034F00005FE7C69F87C07903846083001F038F901
:10350000069900910194079A02920390143F1BA020
:103510000A463B4601F010F901E0FCF7EFFD2D1DD6
:10352000761CD7E705980028C9D1002017B0F0BD58
:10353000252D2A2E732020206F776E65722020683B
:103540006F6C642073757370656E64207468726547
:1035500061640A006D75746578000000202D2D2DC2
:103560002D2D2D2D2D202D2D2D2D202D2D2D2D2DA5
:103570002D2D2D2D2D2D2D2D2D0A0000252D2A2E02
:103580002A7320252D382E2A7320253034642025D7
:10359000640A0000F0B595B00224204601F05EFCFC
:1035A00010A90C72002414940821139108A91191F8
:1035B000001D109029A010212FA201F0BDF800F0ED
:1035C00079FC30A001F0B8F80294204610AC2146F6
:1035D000FFF7AEFD0390267A08AD14980690029985
:1035E00004960698814233DA07912C68271FFCF76E
:1035F00081FD3F78FCF782FD7F203840B04223D127
:1036000005952746143F258AA6680834204601F010
:10361000AFF8A6420ED00095019010211FA00A46D7
:103620003B4601F089F8204602F042FF1F4801F0B6
:1036300083F807E00095019010211DA00A463B4643
:1036400001F07AF8049E059D2D1D0799491CC8E7D5
:1036500003980028BAD1002015B0F0BD252D2A2EE0
:1036600073207620202073757370656E64207468F3
:10367000726561640A00000073656D6170686F7245
:1036800065000000202D2D2D202D2D2D2D2D2D2DD3
:103690002D2D2D2D2D2D2D0A00000000252D2A2E3B
:1036A0002A7320253033642025643A008F7E000879
:1036B000252D2A2E2A7320253033642025640A0004
:1036C000F0B593B00124204601F0C8FB0EA90C729E
:1036D000002412940821119106A90F91001D0E904B
:1036E0003048102130A201F027F800F0E3FB30A0B1
:1036F00001F022F8029420460EAF3946FFF718FD7C
:1037000003903F7A12980590029D04970598854290
:1037100041DAA80006A90E58341FFCF7EBFC21780B
:103720007F220A40BA4232D134462834FCF7E6FC04
:10373000607800903346143B10212DA00A4600F01B
:10374000FBFF21780F200840042804D880002BA11B
:10375000085800F0F1FFF4690020215C401C232987
:10376000FBD0376A391A6420484364303946FCF785
:10377000D3FD03463069F16B726A009101923919E9
:10378000091A23A03A4600F0D7FF049F01E0FCF796
:10379000B5FC6D1CBAE703980028ADD1002013B02A
:1037A000F0BDC0468A7D00087468726561640000DF
:1037B000202D2D2D20202D2D2D2D2D2D2D202D2D6D
:1037C0002D2D2D2D2D2D2D2D202D2D2D2D2D2D2D36
:1037D0002D2D2D20202D2D2D2D2D2D20202D2D2D4D
:1037E0002D2D2D2D2D2D2D202D2D2D0A00000000ED
:1037F000252D2A2E2A73202533642000CE7D000833
:10380000E07D0008E97D0008F27D0008D77D000812
:1038100020307825303878203078253038782020CE
:10382000202025303264252520202030782530388E
:103830007820253033640A00F0B593B00A2420467E
:1038400001F00CFB0EA90C720024129408211191B6
:1038500006A90F91001D0E9025A010212EA200F0A8
:103860006BFF00F027FB2EA000F066FF02942046BD
:103870000EAF3946FFF75CFC0390387A049006AD32
:1038800012980590029C0598844225DA2F683E1F05
:10389000FCF730FC31787F220A4004998A4212D129
:1038A000FCF72CFCB869F969009001913B46143B88
:1038B00010212AA00A4600F03FFFF81E0078C0073A
:1038C00004D12F4803E0FCF719FC02E029A000F026
:1038D00033FF2D1D641CD6E703980028C8D102F0E1
:1038E00013FA014617A000F027FF002013B0F0BD27
:1038F000252D2A2E732020706572696F64696320FC
:10390000202074696D656F75742020202020202090
:10391000666C61670A00000074696D6572000000E2
:10392000202D2D2D2D2D2D2D2D2D2D202D2D2D2DE1
:103930002D2D2D2D2D2D202D2D2D2D2D2D2D2D2DC4
:103940002D2D0A0063757272656E74207469636B45
:103950003A3078253038780A00000000252D2A2ECC
:103960002A73203078253038782030782530387820
:10397000200000006163746976617465640A000068
:103980007D7D00080146002000290FD00A68002A2A
:103990000CD04A68002A09D08868C968884204D0D7
:1039A00001D9421A01E0511A0A18501E7047014607
:1039B000002000290ED00A68002A0BD04A68002A8D
:1039C00008D08B68C968994204D001D9C81A7047D9
:1039D0008818C01A704703460020002B09D0002920
:1039E00007D0002A05D0002006C3186058609860F0
:1039F00001207047E0B500230193009301AB00F074
:103A000004F8002800D001988CBDF0B585B00026E0
:103A1000002845D005460768002F41D06868002877
:103A20003ED000293CD01446002A39D002AA0BC24D
:103A30002846FFF7BCFF002832D0A04202D20A99E4
:103A4000C9072DD1A04200D32046AA6802998E1A38
:103A5000864200D306460446B918039F38460192B1
:103A60003246FCF7E3FB0294A41B05D0B819296881
:103A70002246FCF7DBFB01E00198341868688442B9
:103A800000D30024AC602B69002B03D00021284612
:103A9000029A984701260498002801D002990160F3
:103AA000304605B0F0BDF8B5002400281DD005460D
:103AB0000068002819D06F68002F16D00E46002924
:103AC00013D02846FFF773FF0446B04200D33446B4
:103AD000A8680019C11B00D30846A8602B69002BF9
:103AE00003D000212846224698472046F8BDE0B57D
:103AF00000230193009301AB00F004F8002800D0EC
:103B000001988CBDF0B585B00026002846D005464A
:103B10000768002F42D0686800283FD000293DD0B8
:103B20001446002A3AD002AA0BC22846FFF72AFF01
:103B3000002833D00146A04202D20A98C0072DD1F6
:103B4000A14200D32146EA680298861A8E4200D329
:103B50000E46B8180C46039F394601923246FCF7D0
:103B600065FB0294A41B05D0B91928682246FCF70E
:103B70005DFB01E0019834186868844200D300249A
:103B8000EC602B69002B03D001212846029A98474C
:103B900001260498002801D002990160304605B042
:103BA000F0BD0A2001F00EFFFBE780B500F084FBBA
:103BB000FFF7F7FF80BD0000FEB50446007800283F
:103BC00047D02548006802902448066800270197DE
:103BD00000940298864234D235680622284620494D
:103BE000FCF769FB00282AD12046FCF750FB02466F
:103BF000AD1D20462946FCF75EFB00281FD1019829
:103C0000002803D12846FCF742FB2F4601900024F0
:103C1000385D002806D0295D002903D0884201D1F3
:103C2000641CF5E70FA0294600F086FD0198844248
:103C300000DB04460848006802900194009C0C36A2
:103C4000C7E7002F04D020463946019A01F0D0FB87
:103C5000FEBD00F0EFF8FEBD8C00002088000020C3
:103C6000FB7D000825730A00F0B58BB00D460446B5
:103C7000002D07D02078202801D0092804D16D1EFE
:103C8000641CF5E70020ADE00021C0B2092808D08F
:103C9000202806D08D4203D060184078491CF4E7F4
:103CA00029460191002900D18DE00198801D0090E6
:103CB0004D48006802904D4806680298864200D33D
:103CC00081E03768062238464949FCF7F4FA0028B3
:103CD0000AD1B81D2146019AFCF7EDFA002803D15C
:103CE0000098385C002801D00C36E6E7B0680290F6
:103CF000002868D003A82021FCF7B1FA0022204652
:103D00001646AA4258D20378202B01D0092B08D19D
:103D1000AA4204D200210170521C401CF3E729463C
:103D200000E01146082E35D2A94245D2B200222B1E
:103D300013D1401C03AB985003784A1C222B1AD095
:103D4000AA4218D25C2B05D14378222B02D1401C09
:103D5000891C00E01146401CEEE703AB9850771C2D
:103D60000023C65CCA18092E0DD0202E0BD0AA4203
:103D70000ED25B1CF5E7761CAA421FD2002202700D
:103D80008A1C401CBDE7C018AA423E46B9D315E0C4
:103D90003E4613E017A000F0CFFC03AF1DA501962F
:103DA000002E05D002CF284600F0C6FC761EF7E7AD
:103DB000194800F0C1FC019E002E04D003A9304632
:103DC000029A90470EE02046017820220A43202ADA
:103DD00001D0401CF8E70025057010A0214600F036
:103DE000ABFCE8430BB0F0BD8C0000208800002045
:103DF000FB7D0008546F6F206D616E7920617267E2
:103E0000732021205765206F6E6C79205573653AB9
:103E10000A000000257320008F7E000825733A20D9
:103E2000636F6D6D616E64206E6F7420666F756E6A
:103E3000642E0A00F8B510A000F07EFC1548056855
:103E400015480768164CAF4210D23E68062230462D
:103E50002146FCF730FA002806D17A68B11D11A07E
:103E600000F06AFC0B4805680C37ECE70B4800F0E3
:103E700063FC0020F8BDC04652542D546872656141
:103E800064207368656C6C20636F6D6D616E647324
:103E90003A0A00008C000020880000208F7E000875
:103EA000FB7D0008252D313673202D2025730A0057
:103EB00001207047B0B50F20C54304A4002D04D0E5
:103EC000204600F039FC6D1CF8E7B0BD2D00000065
:103ED000B0B5184C6068002808D000F0E5FB002859
:103EE00005D04F208500FCF705F96051B0BD01F009
:103EF000B3FD0028F5D008340020C143204600F06F
:103F000033FEB0BD10B50B4C6068002808D000F03F
:103F1000CBFB002805D04F2080002058FCF7EEF89E
:103F200010BD01F099FD0028F5D00834204600F0BE
:103F300081FD10BD201E002070B504461F4DE868AD
:103F4000A04204D91EA02649A12200F063F92869E5
:103F5000A04204D823A02249A22200F05BF9608885
:103F6000002804D02AA01E49A32200F053F961685A
:103F7000E8684218A2420FD05388002B0CD12B695D
:103F80009A4209D06969914200D16C6151686160BF
:103F9000231A526882189360A2688318A34202D041
:103FA0005E88002E00D070BD6E69A64200D16B61A4
:103FB000596061684018826070BDC046AC00002046
:103FC0002872745F75696E74385F74202A296D6574
:103FD0006D203E3D20686561705F70747200000066
:103FE000478300082872745F75696E74385F7420A7
:103FF0002A296D656D203C202872745F75696E7486
:10400000385F74202A29686561705F656E640000FE
:104010006D656D2D3E75736564203D3D203000005B
:10402000F0B58DB00893174605910446149B5806C9
:1040300001D55BA000E055A007900122D80600D56D
:104040009343D80701D0302000E020200390980748
:104050000025139904910028069302D4029200953A
:1040600015E0002F07D458070CD4180700250028A6
:10407000F4D5202007E001927F42002002902D20FD
:10408000009007E02B200090002002901546002FA2
:104090001ED001950025002F17D00A26384631463C
:1040A000FCF73AF908990A2902D00F21394001E0BA
:1040B0004643B91B079A515C09AA515508990A2928
:1040C00000D038096D1C0746E5E70198089004E028
:1040D000089509A83021017001251298049FBD425E
:1040E0002946059E00DC3946401A1123069A1A42D9
:1040F00001D0039B12E0002801DC002300E0012333
:10410000089A1A40801A039B012806DBB44201D2A8
:1041100020222270401E641CF6E7401E029A002AEC
:1041200005D1B44201D2009A2270641C401E069A46
:10413000D2060FD4012805DBB44200D22370401E02
:10414000641CF7E7401E05E0B44201D23022227021
:10415000491E641C8D42F7DB08E0B44204D209A971
:104160004919491E097821706D1E641C002F08D062
:10417000002DF2DC05E0B44201D220212170401E66
:10418000641C0128F7DA20460DB0F0BD303132331F
:104190003435363738396162636465660000000083
:1041A000303132333435363738394142434445466D
:1041B000000000001CB514200A210091019001208C
:1041C000830208A00949002201F022FA04460028CF
:1041D00004D107A00AA1C52200F01CF8204601F076
:1041E00075FC1CBD6D61696E00000000AB3B0008F2
:1041F00074696420213D2052545F4E554C4C0000A0
:1042000072745F6170706C69636174696F6E5F690D
:104210006E6974001CB513460A46014601A80024C5
:10422000047008480468002C04D0084611461A4659
:10423000A0471CBD04A000F07FFA01A80078002868
:10424000FBD01CBDF40F0020282573292061737357
:10425000657274696F6E206661696C656420617453
:104260002066756E6374696F6E3A25732C206C69D5
:104270006E65206E756D6265723A2564200A0000D5
:10428000B0B504464C43204600F07CFA05460028B1
:1042900004D000212846224600F080FB2846B0BD0D
:1042A000B0B5044C094DAC4202D201CC8047FAE7CC
:1042B000B0BDC0466C860008B0B5044C044DAC429D
:1042C00002D201CC8047FAE7B0BDC0467486000830
:1042D0009886000880B5FBF70DFF0F494A88521CED
:1042E0004A80FBF70BFF80BD10B5FBF703FF0A4CBC
:1042F0006188491E618009B2002902DDFBF7FEFEDC
:1043000010BD00216180FBF7F9FE60680028F7D03E
:1043100000F03EFE10BDC046F4000020F0B585B0B0
:1043200000287CD00446FBF7E5FE06468B2085007E
:1043300000F0BAF9002809D03A483B4F394600F05E
:10434000FBF93A4839462A46FFF764FF3046FBF747
:10435000D5FEA00704D0AA1C35A03349FFF75AFFA9
:104360003F4EF068A04202D83069A04204D82A1D0E
:104370003C482D49FFF74EFF7168002901D02046C7
:104380008847F068A0424AD83069A04247D90195D1
:104390003046203000210391C943049000F032FFE1
:1043A00027460C3FF520410125460A3D2888002874
:1043B00002D0388888421DD002912BA000F0BCF9B1
:1043C0003B882A882FA0394600F0B6F928880028B3
:1043D00005D1019A223237A01349FFF71BFF388815
:1043E0000299884206D0019A233235480E49FFF7D8
:1043F00011FF02993980039828807069874200D2A2
:104400007761F068083C21680818381AB1694018CB
:10441000B0613846FFF790FD049800F0AFFE05B09C
:10442000F0BDC046337E00083F830008708200085C
:1044300028282872745F75626173655F7429726DD4
:10444000656D292026202852545F414C49474E5F14
:1044500053495A45202D20312929203D3D20300047
:10446000AC000020A0820008746F20667265652091
:104470006120626164206461746120626C6F636BAF
:104480003A0A00006D656D3A203078253038782C76
:10449000207573656420666C61673A2025642C2062
:1044A0006D6167696320636F64653A2030782530F9
:1044B00034780A006D656D2D3E75736564000000EB
:1044C0007282000880B502F0EFFA02F01DF87D203C
:1044D000C1000C480068FBF71FFF401E010E08D109
:1044E000094948600948FF2202700720086000203F
:1044F0008860FDF73DFAFFF7D3FE0548054900F057
:104500008DFF80BD0C00002010E000E023ED00E0F6
:10451000682400200040002080B5FDF71BFAC0B2DF
:1045200080BD000080B50246002002A1FDF7C0FA60
:1045300080BDC046257300000446C1690FA0134D1D
:10454000A847A16912A0A847616915A0A8472169D9
:1045500017A0A847E1681AA0A847A1681CA0A8470F
:1045600061681FA0A847216821A0A84724480168C6
:1045700024A0A847FFF7A4F8FEE7C0467073723A7C
:10458000203078253038780A0000000039470008CC
:104590002070633A203078253038780A0000000017
:1045A000206C723A203078253038780A00000000FC
:1045B0007231323A203078253038780A0000000015
:1045C0007230333A203078253038780A0000000005
:1045D0007230323A203078253038780A00000000F6
:1045E0007230313A203078253038780A00000000E7
:1045F0007230303A203078253038780A00000000D8
:10460000F800002068617264206661756C74206F28
:104610006E207468726561643A2025730A00000098
:10462000F0B5141D072294432246403A3F25ED433E
:104630000D4E002D02D066512D1DFAE725461C3D7A
:1046400000262746203F39602E606E60AE60EE6027
:10465000211F01252D060D602146083908600C3CFC
:1046600023601046F0BDC046EFBEADDE10B5E120C0
:10467000400200242146FDF779FC4B2080012146B1
:10468000FDF780F8204610BD10B5FBF733FD04465A
:1046900012480178491C01704068002800D080470A
:1046A0002046FBF72BFD10BD10B5FBF723FD0B4992
:1046B0000C78FBF723FD204610BDC04610B5FBF774
:1046C00019FD044605480178491E017080680028DC
:1046D00000D080472046FBF711FD10BDA000002050
:1046E00080B500681C3801F075F980BD70B51646BC
:1046F0000C460546084601F03DFA002E14D0012E66
:1047000019D121463D3128460068A8420CD021220B
:10471000825C0B789342F7D2416822461C320A60D1
:10472000E0612162426070BD686821461C31016011
:10473000E5612062696070BD83B0B8B5044605A824
:104740000EC005AB0093064DFF212846224601F01E
:10475000DFFC2846FFF7E6FEB8BC01BC03B000470B
:104760000010002080B5002801D0FFF7DBFE80BDDF
:104770000021C9430246491C12688242FBD1084607
:1047800070470000F0B587B00027002853D00446DA
:10479000FBF7B0FC0546FFF787FF00280AD0574813
:1047A000574E3146FFF7C8FF2320C2005548314617
:1047B000FFF730FD2846FBF7A1FCE41C03208443EF
:1047C000514DA868844236D82846203000210491F3
:1047D000C943059000F016FD0C2C00D80C24A968E4
:1047E000E868069402910B1B696903910F1A0699F8
:1047F0009F421CD23D46C61977687288002AF7D1BD
:104800002A460C32BC1A8C42F2D306990B460C3362
:104810000193F5235B01049318318C420ED2019C65
:10482000012272807A1B384DAB699A181EE00598F8
:1048300000F0A4FC049F384607B0F0BD069952185A
:104840000499815283185F6000245C8072609D60CF
:10485000012474805B68029C0C34A34201D0C3180D
:104860009A60294DAA6901990C468A18AA61EB69D8
:104870009342039900D2EA61049A32802322D7003E
:104880008E4213D12A694B88002B05D0914203D068
:10489000496841186961F6E7914207D0002B05D0BD
:1048A0003A466A3219A01649FFF7B4FC059800F0A1
:1048B00065FCA019296988423C4605D922466E321A
:1048C0001C480F49FFF7A6FC37460C37B80705D040
:1048D00022466F3218480A49FFF79CFCB00705D002
:1048E000703416A006492246FFF794FC2A68002A75
:1048F000A1D03846069990479DE7C046337E000810
:104900009682000870820008AC00002028286C669F
:10491000726565203D3D20686561705F656E642944
:10492000207C7C2028216C667265652D3E75736540
:1049300064292900FC82000829820008282828729E
:10494000745F75626173655F74296D656D292026DA
:10495000202852545F414C49474E5F53495A4520E5
:104960002D20312929203D3D2030000010B5814205
:104970000AD28B18834207D9491E431E002A0CD045
:104980008C5C9C54521EF9E70346002A05D00C7833
:104990001C705B1C491C521EF7E710BD10B5042AA1
:1049A00014D30323034011D1CBB20C4C5C43034618
:1049B0000F2A08D91C605C609C60DC60103A1033E0
:1049C000F6E710C3121F042AFBD204E0034602E0FC
:1049D00019705B1C521E002AFAD110BD01010101A1
:1049E000F8B514460E46054607462637002804D17A
:1049F0000A480BA10E4AFFF70DFC03212846324658
:104A000000F05AFA0020A8620121A98429461C312D
:104A1000E9612962FF2139806C74F8BDE97E0008E4
:104A200072745F6D757465785F696E6974000000FB
:104A30001D020000F8B50446CB208500002C04D1EF
:104A40009E4846492A46FFF7E5FB204600F01AFA41
:104A5000032804D06A1C9A484049FFF7DBFBFBF7A8
:104A600049FB064600F0F8FF002809D191483B4F6A
:104A70003946FFF761FEAA1DBC483946FFF7CAFB5D
:104A8000FBF738FB0746FFF70FFE002808D0B548B4
:104A90003249FFF751FEAA1DB4483049FFF7BAFB6F
:104AA0003846FBF72BFB3046FBF728FB00F0D4FF22
:104AB0000746FBF71FFB054629480168002901D07E
:104AC00020468847A06A874207D00220C043841C42
:104AD000BC632846FBF712FB0AE0264626367078B0
:104AE000401E7070000605D02846FBF707FB002427
:104AF0002046F8BD3D20385C3178814204D0022147
:104B00003846324600F032FDE16920461C308142D1
:104B100012D00A461C3AA2622122895C3170717857
:104B2000FF290DD0491C7170FFF7DAFD2846FBF70D
:104B3000E5FA00F02DFADAE7A08C0A49884205D19F
:104B40002846FBF7DBFA0220C443D1E70021A1622B
:104B5000FF213170401CA084C6E7C046877F000853
:104B600008110020FFFF0000FEB5044601910291EC
:104B7000FBF7C0FA07465320C60000F06DFF00287F
:104B800009D14C484C4D2946FFF7D6FD77482946B8
:104B90003246FFF73FFBFBF7ADFA0546FFF784FD12
:104BA000002808D06F484449FFF7C6FD6F484249C6
:104BB0003246FFF72FFB2846FBF7A0FA3846FBF7F3
:104BC0009DFA002C04D1F21C3C483B49FFF722FB24
:104BD000204600F057F9032804D0321D38483649E2
:104BE000FFF718FB00F038FF0746FBF783FA05468E
:104BF00034480168002901D02046884721462631E3
:104C00000026BE63A06AB84208D0A28C002A1CD03D
:104C1000A762501EA0843D20385C08704878FF28A9
:104C200005D12846FBF76AFA0220C5430BE0401C79
:104C300048702846FBF762FA23480168002901D032
:104C40002046884735462846FEBD0199002929D0CF
:104C500000953D21425C795C914204D23A463D3256
:104C6000022100F083FC627C20461C303946FFF7AD
:104C70003DFD0198012809DB3D465435002102AA7B
:104C8000284601F0B3F8284601F082F90098FBF7B6
:104C900035FA00F07DF9BD6B002DD4D1FBF72AFA6F
:104CA0000546C6E70220C14328464D1CBD63FBF7FD
:104CB00025FAC8E75A7E0008257F0008E97E00082B
:104CC000A4810008101100200C110020F8B50091FB
:104CD0000546FBF70FFA0646C3204700FFF7E4FC42
:104CE000002809D01F48204C2146FFF725FD1F480A
:104CF00021463A46FFF78EFA3046FBF7FFF9284681
:104D000000F0ACF80646002804D13A1D8A4816493E
:104D1000FFF780FAF068FFF735FD074600281ED040
:104D2000F268002438462146FFF738FE7C743D7453
:104D300010223846009900F05BFB85480168002985
:104D400001D038468847FBF7D5F9716879613A4652
:104D500014324A607260311DB961FBF7CFF93846F1
:104D6000F8BDC046337E00089E83000870820008AC
:104D700010B50446002805D1DD204200134814492F
:104D8000FFF748FA10202056002806D5DD20400005
:104D9000421C10A00E49FFF73DFA2F480168002978
:104DA00001D02046884700202074FBF7A3F96169F1
:104DB000A2694A60A2691160214614316161A16152
:104DC000FBF79CF92046FFF7A9FA10BD7D83000888
:104DD000B183000821286F626A6563742D3E74797F
:104DE000706520262052545F4F626A6563745F438A
:104DF0006C6173735F537461746963290000000010
:104E000010B50446002805D1B32042000C480DA17E
:104E1000FFF700FA10480168002901D020468847B2
:104E200000202074FBF766F96169A2694A60A269F3
:104E30001160214614316161A161FBF75FF910BD7A
:104E40007D83000872745F6F626A6563745F646576
:104E500074616368000000000411002010B57F2118
:104E6000CB4307491A46103208D0CB1880241B5D6B
:104E700083421346F7D18818703010BD002010BD52
:104E80001000002010B50446002805D1FF22F032A2
:104E9000034804A1FFF7BEF9217C7F20084010BD24
:104EA0007D83000872745F6F626A6563745F676513
:104EB000745F747970650000FEB50292044601913A
:104EC0000846FFF7CBFF0546FF273437002804D1FB
:104ED00019481A493A46FFF79DF9FFF7FBF92E1DCD
:104EE00035462D68B5420AD028461438A042F8D17C
:104EF0003A46103212A01149FFF78CF9F1E78020F1
:104F0000019D0543FFF7F0F9257410222046029910
:104F100000F06EFA0E480168002901D0204688474B
:104F2000FBF7E8F831686161224614324A6032606A
:104F3000A661FBF7E3F8FEBD66830008C2830008A4
:104F40006F626A20213D206F626A65637400000011
:104F50000011002010B50446002805D177208200FA
:104F6000034804A1FFF756F9207CC00910BDC046D4
:104F70007D83000872745F6F626A6563745F697332
:104F80005F73797374656D6F626A656374000000A6
:104F9000F8B5FBF7AFF804464D4F7888002803D0EA
:104FA0002046FBF7ABF8F8BDF868FDF739FB401E6B
:104FB000C100464A555829461C397E68B142EFD097
:104FC00079603870BA68002A01D0304690470835B9
:104FD000243607480078002804D030462946FBF7DD
:104FE00090F8DDE730462946FBF78BF8D8E7C04656
:104FF000A0000020F8B5044605463C35002805D140
:10500000FF2218320E480FA1FFF704F9FBF772F8E0
:105010006978C9002D4A51184A68226223461C3318
:105020001360226C2A4EF7681743F7602A78F0263F
:105030001640721C2A704B60E161FBF75FF8F8BD07
:10504000D183000872745F7363686564756C655F13
:10505000696E736572745F746872656164000000E4
:1050600010B50446002805D1FF2246320F4810A192
:10507000FFF7D0F8FBF73EF8E169226A4A60226A3E
:10508000116021461C31E16121623D21615CC90052
:105090000E4A53185158994204D1216C0C4AD368D6
:1050A0008B43D360FBF72AF810BDC046D1830008BC
:1050B00072745F7363686564756C655F72656D6F4C
:1050C00076655F74687265616400000018110020E5
:1050D000F4000020F8B516460D460090FBF70AF8DC
:1050E0000446FF270E37FFF7DFFA002808D0EE4806
:1050F0000F49FFF721FBEE480D493A46FFF78AF8C2
:105100002046FAF7FBFF280C04D07A1C1A480849FD
:10511000FFF780F802200099FFF7D8FD002805D09E
:105120008584467401461C31C1610162F8BDC046E8
:10513000A57F0008F8B51C4616460F460546002810
:1051400004D171480B49D222FFF764F8300C04D027
:1051500009480849D322FFF75DF8022128463A465C
:10516000FFF7AAFEAE8428461C30E86128626C7402
:105170000020F8BD24810008FA7E0008F8B5044636
:10518000002805D1FF22B8325F481B49FFF742F8DB
:105190002046FFF777FE022806D0FF20B830421CD9
:1051A0005B481549FFF736F814480168002901D01B
:1051B0002046884725461C35FAF79CFF0646E769D6
:1051C000AF4203D02846FFF78BFA0BE0A08C0C49C6
:1051D000884205D13046FAF791FF0220C44309E026
:1051E000401CA0843046FAF789FF0024AF4201D06A
:1051F000FFF7CEFE2046F8BD787F0008081100209A
:10520000FFFF0000FEB50D460446029153208700C3
:10521000002C04D13C483D493A46FEF7FBFF2046AE
:10522000FFF730FE022804D07A1C39483749FEF7D0
:10523000F1FF38480168002901D020468847FAF775
:1052400059FF0646A08C00280CD0401EA084304692
:10525000FAF754FF314801680025002951D0204653
:1052600088474EE0002D47D0FAF744FF019000F048
:10527000F3FB002809D128482449FFF75DFA3A4694
:1052800021328B482149FEF7C5FFFAF733FF009022
:10529000FFF70AFA002809D083481C49FFF74CFAA7
:1052A0002137834819493A46FEF7B4FF0098FAF7C8
:1052B00025FF0198FAF722FF00F0CEFB07460020F9
:1052C000B863627C20461C303946FFF70FFA012D87
:1052D00009DB3D465435002102AA284600F086FD30
:1052E000284600F055FE3046FAF708FFFFF750FE5B
:1052F000BD6B002D05D1ADE73046FAF7FFFE01206A
:10530000C5432846FEBDC046A97E0008197F000897
:10531000337F0008101100205A7E00080C11002075
:105320001CB507A0094CA04709A0A04711A00090F8
:1053300013A0032101220523A04719A0A0471CBDEB
:105340000A205C207C202F0A00000000394700085A
:105350002D205254202D2020202020546872656179
:1053600064204F7065726174696E6720537973743D
:10537000656D0A00536570202034203230323400CD
:10538000202F207C205C202020202025642E2564D6
:105390002E2564206275696C642025730A00000064
:1053A0002032303036202D203230323020436F70A2
:1053B0007972696768742062792072742D746872DA
:1053C000656164207465616D0A00000081B0C0B53C
:1053D000039303AB009300F09BFE88BC02BC01B0BA
:1053E00008470021425C491C002AFBD1481E704737
:1053F00010B5002A09D003460C781C70002C05D08B
:105400005B1C521E491C002AF6D110BD01218A42A4
:10541000FBD000245C54491CF9E70000F8B50F46A6
:1054200000900320C5430C462C40FAF763FE064665
:10543000FFF73AF9002808D01B481C49FFF77CF910
:105440001B48D2221949FEF7E5FE3046FAF756FE10
:10545000192C009905D3C81C28402246183A8242CC
:1054600004D218A03A46FFF767F9F8BD211A0A4698
:10547000183A104DAA60F52252010C39002302603F
:10548000416083600C3C6160E8602C610A482060E8
:10549000A8680C30A0602846203008A10122FFF740
:1054A00049FEE8686861F8BD337E00085283000851
:1054B00070820008AC000020A01E010068656170C9
:1054C000000000006D656D20696E69742C206572A6
:1054D000726F7220626567696E20616464726573C1
:1054E0007320307825782C20616E6420656E6420EE
:1054F0006164647265737320307825780A00000057
:105500001348002141802022124B002A04D01B6046
:105510005B600833521EF8E741601F2202700246AA
:105520001032C160026142617047C04610B5084C3C
:10553000E068FDF775F8C0000649401808380068B3
:1055400001461C3961600830FAF713FE10BDC046F1
:10555000F400002018110020024801460C31C160FF
:10556000016170470C01002070470000F8B5154636
:105570000E460446002804D191482349234AFEF7E9
:1055800049FE2046FFF77EFC012805D01F48421C3B
:105590008D481D49FEF73EFE002E19D0012E1BD06E
:1055A000022E2ED127463C37FAF7A4FD064638785E
:1055B0000F210140012918D12046FFF751FD28781D
:1055C00078700121814021642046FFF713FD11E02E
:1055D000204600F07BFA14E02046FFF7BBFC0128D0
:1055E0000CD1204600F0A0F80BE02878787001215B
:1055F000814021643046FAF781FD02E0204600F048
:105600002DF80020F8BDC046808400087702000015
:10561000F0B585B01F4604920D4601460120FFF704
:1056200055FB0024002815D006463846FFF7AAF897
:1056300000280CD003460B980A990097019102901C
:1056400030462946049AFDF755F8344602E03046C4
:10565000FFF78EFB204605B0F0BD000070B5044694
:10566000CF204500002C04D11D481E492A46FEF7D4
:10567000D1FD2046FFF706FC012804D06A1C1A4819
:105680001849FEF7C7FD2046FFF764FC002804D048
:10569000AA1C16A01349FEF7BDFD3C20215C0F207B
:1056A000084004D0042819D02046FFF7D9FC25462D
:1056B0003C352046FDF77AF82046543000F0ECFBEC
:1056C00026461C36FAF716FD8E490A6856600423F2
:1056D0002B700E60E2612162FAF710FD002070BDB0
:1056E000D183000848840008E383000872745F6F68
:1056F000626A6563745F69735F73797374656D6FF4
:10570000626A656374282872745F6F626A65637485
:105710005F742974687265616429203D3D2052548C
:105720005F46414C53450000B0B50446FF253A356D
:10573000002804D1224823492A46FEF76BFD204663
:10574000FFF7A0FB012804D06A1C1F481D49FEF783
:1057500061FD2046FFF7FEFB002804D1AA1C1BA018
:105760001849FEF757FD3C20215C0F20084004D06B
:10577000042822D02046FFF773FC25463C352046FE
:10578000FDF714F82046543000F086FB0420287002
:105790002046FFF7DFFB012803D12046FFF730FB4F
:1057A0000BE025461C35FAF7A5FC56490A685560FA
:1057B0000D60E2612162FAF7A1FC0020B0BDC04695
:1057C000D183000859840008E383000872745F6F76
:1057D000626A6563745F69735F73797374656D6F13
:1057E000626A656374282872745F6F626A656374A5
:1057F0005F7429746872656164290000B0B5DC4883
:105800000568FAF777FC04462846FCF7CFFF2846E0
:10581000FFF726FC3C20042129542846543000F090
:105820003BFB2846FFF796FB012803D12846FFF7EC
:10583000E7FA07E0334801682A461C324A600260F2
:10584000E9612862FFF7A4FB2046FAF757FCB0BDD8
:105850000024074D2646042E06D0B0002858002804
:1058600000D08047761CF6E700F004F8F2E7C04667
:10587000600F002070B5FAF73DFC0446FEF714FFF8
:10588000002809D013A01D4D2946FEF755FF1CA086
:1058900093222946FEF7BEFC1A4E2046FAF72EFC4C
:1058A000FAF728FC04463568B5420ED003CD4160B6
:1058B000083D696808602D606D606869FEF72EFD1F
:1058C0001C3D2846FFF754FAE7E72046FAF716FC96
:1058D00070BDC04646756E6374696F6E5B25735DFF
:1058E000207368616C6C206E6F7420626520757324
:1058F000656420696E204953520A00001D7E00082D
:1059000030000000040100201FB5202003901F205C
:10591000029008480090012000020190064C07A167
:10592000084A0023204600F00FF8204600F0CEF889
:105930001FBDC0461C120020D00E00207469646C8C
:105940006500000051580008F0B587B00693059235
:105950000A4607460C9E002806D1124812491446F2
:10596000E922FEF757FC22460F9804900E9C0D9DED
:10597000002E06D10DA00C490392EA22FEF74AFC44
:10598000039A01213846FFF797FA0095019404988D
:10599000029038460599069A3346FCF7ABFE002084
:1059A00007B0F0BDD1830008B4840008737461634C
:1059B0006B5F737461727420213D2052545F4E55A9
:1059C0004C4C000080B500F09BF900F049F8002035
:1059D00080BD000070B50446002804D19F481B49D3
:1059E0001B4AFEF717FC2046FFF74CFA012805D0AA
:1059F0001748421CAA481549FEF70CFC3C20205CC5
:105A00000F210140002502291CD1FAF773FB06463D
:105A1000E069216A4160216A086020461C30E0612B
:105A200020622046543000F035FB3046FAF766FB22
:105A30002046FFF7DFFA07480168002903D0204617
:105A4000884700E0ED43284670BDC0463784000813
:105A5000F702000018120020A74800687047C046EF
:105A6000F8B50090FAF746FB0546A3480468002CF9
:105A700005D1FF22FC3279481349FEF7CBFB2046C3
:105A8000FFF700FA012806D0FF20FC30421C8448B2
:105A90000D49FEF7BFFB204600F06CF8274654374F
:105AA00000266A463846314600F0A0F9384600F034
:105AB0006FFA2846FAF722FBFFF76AFAA06B801C00
:105AC00000D1A6630020F8BD9284000870B504469A
:105AD000FF250E3506463C36002804D114481549EA
:105AE0002A46FEF797FB3078000704D06A1C12A004
:105AF0001049FEF78FFB2046FFF7C4F9012804D0B8
:105B0000AA1C67480B49FEF785FB02203070B0786D
:105B100070700121814021642046FFF75BFF7648C9
:105B20000068002801D0FFF733FA002070BDC0469E
:105B3000D1830008A2840008287468726561642D0E
:105B40003E7374617420262052545F54485245417C
:105B5000445F535441545F4D41534B29203D3D20F8
:105B600052545F5448524541445F494E49540000E5
:105B7000F8000020F8B50446002804D137481A4937
:105B80001A4AFEF747FB2046FFF77CF9012805D0AB
:105B90001648421C42481449FEF73CFB3C20205C5E
:105BA0000F210140002501291AD127463C37FAF779
:105BB000A1FA06462046FFF753FA3878F021014053
:105BC000881C38702046543000F064FA3046FAF7EA
:105BD00095FA07480168002903D02046884700E06D
:105BE000ED432846F8BDC04625840008CD020000DC
:105BF0001C130020B0B50446174D002804D11748E7
:105C000017492A46FEF706FB3C20205C0F21014085
:105C1000022904D06A1C13A01149FEF7FBFA2046A2
:105C2000FFF730F9012804D0AA1C1D480C49FEF7E3
:105C3000F1FAE069216A4160216A08600120C043ED
:105C4000A06320461C30E06120622046FFF7D2F9B5
:105C5000FFF79EF9B0BDC04623030000D1830008C2
:105C6000C3840008287468726561642D3E73746192
:105C70007420262052545F5448524541445F535487
:105C800041545F4D41534B29203D3D2052545F54B8
:105C900048524541445F53555350454E440000001F
:105CA000E3830008B0B5FAF725FA134909683C22E6
:105CB0008A5C0F231340012B19D1CA690B6A9A42DF
:105CC00015D00C463C340D461C3553600B6A0D62F2
:105CD0001A606278D200094B9A1853681D60CA6135
:105CE0000B625560FAF70AFAFFF752F901E0FAF78A
:105CF00005FA0020B0BDC046F800002018110020B1
:105D0000C1170843704700000A4800687047C04642
:105D100080B508480168491C0160FFF79DFE016DD0
:105D2000491E016503D1C16C0165FFF7BBFF00F09F
:105D300003F880BD24130020FEB501A80190029055
:105D4000FFF7E2FF0646FAF7D5F90090D048C5689C
:105D50000C30854243D06869301A234988423ED8C6
:105D60002C461C3CCA480168002901D020468847BF
:105D700003CD4160083D696808602D602F460B3FE8
:105D80003878810702D4FE210840387001984560B8
:105D9000286001A868600195A968E8688847FFF74E
:105DA000B3FF0646BA484168002901D0204688471B
:105DB00001A801998142C9D003CD4160083D6968BD
:105DC00008602D606D6038788107BFD5C107BDD0F0
:105DD000FE2108403870204600F0DAF8B6E7009857
:105DE000FAF78CF9FEBDC046FEFFFF7F70B5154681
:105DF0000E460446002805D1FF22DA32C048194970
:105E0000FEF708FA2046FFF73DF80A2806D0FF20E3
:105E1000DA30421CBC481349FEF7FCF9FAF76AF97C
:105E2000042E1BD87E4436797600B744020A0C1043
:105E300005002968E16211E0617CC9070CD10021ED
:105E40000BE0E16A09E0617CFD220A4002E0617C2E
:105E500002220A43627401E001212960FAF74EF937
:105E6000002070BD0685000870B51C4615460E461C
:105E700001460A20FEF72AFF00280CD004990022D0
:105E8000FE230B40437401461C31C161016246622E
:105E90008562C462026370BD10B50446002804D157
:105EA00017481849DD22FEF7B5F92046FEF7EAFF4C
:105EB0000A2804D014481349DE22FEF7ABF9204625
:105EC000FFF748F8002804D110A00E49DF22FEF7A2
:105ED000A1F9FAF70FF9E169226A4A60226A1160B2
:105EE000617CFE220A40627421461C31E16121621C
:105EF000FAF704F92046FEF783FF002010BDC046E4
:105F0000D5840008F68400082585000872745F6F48
:105F1000626A6563745F69735F73797374656D6FCB
:105F2000626A656374282674696D65722D3E7061BE
:105F300072656E7429000000FEB5029301920F464F
:105F40000546099E089C002804D10C480CA1C922D2
:105F5000FEF760F90A2128463A46FEF7ADFF002019
:105F6000FE210E406E7429461C31E96129620199B7
:105F700069620299A962EC622863FEBDD5840008BB
:105F800072745F74696D65725F696E697400000098
:105F9000FEB50446FF264236002804D12E482F497C
:105FA0003246FEF737F92046FEF76CFF0A2804D088
:105FB000721C2B482949FEF72DF9FAF79BF802903D
:105FC000E069216A4160216A0860607CFE2101402D
:105FD000617420461C30E061019020622148016814
:105FE000002901D020468847E06A1F4DA84205D30A
:105FF00010361EA019493246FEF70CF9FFF784FE51
:10600000E16A0A182263224801460C31036901261D
:10601000F0070DD008460026984207D001460068D8
:106020004769BF1AF7D0AF42F5D2F1E71946EFE75B
:106030000868E061019A4260154B9868401C9860BE
:106040000A602162607C0121014361740298FAF7C1
:1060500055F80020FEBDC046D584000861850008C3
:10606000258500080C110020FFFFFF7F74696D6516
:10607000722D3E696E69745F7469636B203C2052B7
:10608000545F5449434B5F4D4158202F203200004C
:106090000C010020B0B50446002805D1DB204200E9
:1060A00017481849FEF7B6F82046FEF7EBFE0A2817
:1060B00006D0DB204000421C13481249FEF7AAF824
:1060C0000025607CC00701D1ED4316E00F48016850
:1060D000002901D020468847FAF70CF8E169226AC6
:1060E0004A60226A1160617CFE220A406274214685
:1060F0001C31E1612162FAF701F82846B0BDC046C3
:10610000D58400081785000825850008081100209F
:10611000F0B58DB00B9304460C9200230893DF4337
:1061200005910029069701D405996718E143039169
:10613000049407971078252807D0002800D133E170
:10614000BC4200D22070641C2AE1501C089F0178D8
:10615000202909D0232909D0302909D02D2909D097
:106160002B290BD1042106E0082104E0202102E0C4
:10617000012100E010210F43401CE8E70C900A4683
:10618000303A092A05D80CA800F0ACF906460C985C
:106190000DE02A290AD1401C0C900B9940C9002E11
:1061A0000B9104D510210F43764200E0069E037840
:1061B0002E2B0CD1411C0C9142781346303B092BFD
:1061C00009D80CA800F08EF902460C990CE00146A3
:1061D00006980A900CE02A2A05D1811C0C910B9894
:1061E00004C80B9000E0069AD01782430A920B78FD
:1061F000042018436C2805D1481C0C904A780146AD
:10620000184601E000201A4615466F3D0A23092D65
:1062100017D9252A5BD0582A5FD0692A1FD0642A53
:106220001DD0632A20D1F80600D5A2E0079F022ED8
:1062300000DAA0E0BC4201D220202070761E641C4F
:10624000F5E709930346C0467D442D796D00AF44C0
:10625000041B0B0B300B490B0B47082041E0099343
:106260000346022007433DE0079FBC4203D225209E
:1062700020700C990A78601C002A00D18DE0B84289
:1062800000D20270A41C8BE00B9804C80B900A98F3
:106290000190701C00D108260096414241410F43F5
:1062A000F8B2029010232046079F3946FDF7B8FE4A
:1062B00075E00B9A02CA002900D144A100230B9279
:1062C0009E422BD0C85C002829D05B1CF8E7079FB2
:1062D000BC4200D337E7252034E70346402007437C
:1062E00010200990682B04D06C2B0B9D2A68099B09
:1062F00006E00B980288B807099B00D512B20B9DE7
:10630000F8B200960A99019102902046079F3946FB
:10631000FDF786FE04462D1D0B9541E033460A9895
:106320008342024600DC1A46002800DC1A46F806C2
:1063300009D4079FB24208DABC4201D22020207063
:10634000761E641CF6E7079F00E0761E0023E01827
:1063500093420BDAB84201D2CD5C05705B1CF6E7C4
:10636000B84201D220210170761E401CB242F7DBF8
:1063700015E0079F00E0761E0B99BC4201D2086829
:106380002070091D641C022E05DBBC4201D22020B6
:106390002070761EF6E70B9102E0491E0C91044630
:1063A0000C98421C0C92C5E605980028039900D46D
:1063B0000146002905D0BC42204600D3781E08992A
:1063C00001700498201A0DB0F0BDC046284E554CFF
:1063D0004C29000010B501218A02184803460C3BE5
:1063E0001C6814431C6000BF00BF00BF0A071C6884
:1063F00014431C6000BF00BF00BF0A02104B1C68A2
:1064000014431C60036802241C43046003681024C6
:106410001C4308239C43046003680B430360036828
:106420005B07FCD503231B0204689C4314430460F0
:10643000C90302680A43026010BDC0464010024012
:106440000070004000207047002070470020704717
:106450000020704780B5F9F74DFEFEF733F8FEF7E0
:106460005FFFFFF779F8FFF74BF8FDF7A3FEFFF7A3
:106470007BF8FFF749FAFFF759F8002080BD0000CC
:1064800010B5044606A0FEF757F9FCF75FFADF20C7
:106490004000221804480549FEF74EF910BDC046D9
:1064A0001B5B324B0D000000187E000838070020EF
:1064B000F8B5044609A50AA607463F68A7420BD0CF
:1064C00039461C392846FEF737F93868A042F4D01F
:1064D0003046FEF731F9F0E7F8BDC04625730000FD
:1064E0002F00000010B5026800211378303B092B03
:1064F00008D8531C03600A244C43117861183039C2
:106500001A46F2E7084610BD0448016804220A430F
:106510000260016801220A430260704710E000E057
:10652000B0B5026814215143154A8C580A4B2340D8
:106530004468C568254304692C434569254384693B
:106540002C431C438C508B581F242404A343806885
:10655000000418438850B0BD0FE7FFFF10B5016875
:1065600014224A4306495318C4685C6044689C601E
:106570008068D860505801230343535010BDC04673
:1065800008000240F8B50D4606460524204600F0F6
:1065900021F8002800D0F8BD284F38680621009166
:1065A000884330433860022E07D17F2000023968CB
:1065B000814328020843386000E03224386808210B
:1065C00001433960204600F005F83968009A91438C
:1065D0003960F8BD10B50446F34800687D21C90054
:1065E000F9F79AFE6043411C07480268D20303D5BD
:1065F000491EFAD1042010BD0168044A02601C2023
:106600000840411E884110BD102002401C000001BE
:10661000F8B50D46064601242046FFF7DBFF0028AB
:1066200000D0F8BD054F38682043386035602046FB
:10663000FFF7D0FF3968A1433960F8BD142002404C
:10664000FEB50D4601900024019E29680846E040F1
:106650002CD00120A040014026D0084648436A685B
:10666000034653430327474302942C463568BD43F2
:106670001D433560A3684343F568BD431D43F56082
:106680002546029C022A0FD12A69FF2909D84043D6
:1066900042430F214143019B186A8843104318620B
:1066A00002E0019800F00EF8641CCEE76868401E16
:1066B000012806D8E8684843019B5A688A43024388
:1066C0005A60FEBD090A494349434A430F234B43DD
:1066D000416A994311434162704770B50E460446C2
:1066E00000680125A8432060280321688143F068E1
:1066F000084320600320410222688A4371691143E4
:106700002160010362688A43316911436160E16A73
:106710000F22914332680A43E2620002A16881437A
:10672000B0690843A060B168204600F01BF800285B
:1067300015D120680C2188437168014321602068CD
:10674000216801220A432260010702D5E16989021A
:10675000FCD50025400702D5E0694002FCD528465B
:1067600070BD000070B50D460446002621488442E5
:106770000ED02148844230461ED1204800680005D2
:10678000810F1F487944097949008F440D10151372
:106790001A4800688005810F1948C0467944097974
:1067A00049008F440104090700F048F804E000F0B4
:1067B00081F801E00120C003E16A0907C90E11A2B6
:1067C000515AF9F7A9FD010E00026A0880187141BB
:1067D0002A463346F9F7FAFC10494118104A91420B
:1067E00006D8E1680F4A0A400243E260002070BD0B
:1067F000012070BD00840040008000403C10024039
:106800000024F400010002000400060008000A0051
:106810000C001000200040008000000100FDFFFF80
:10682000FFFC0F000000F0FF80B500F043F8BC490A
:1068300009684905490FC84080BDC04610B507200A
:106840000403FFF7F1FFB64909682140090B03294A
:1068500001D3C91E00E00021C84010BD10B50720BB
:106860000404FFF7E1FFAE4909682140090C032940
:1068700001D3C91E00E00021C84010BD10B50C4C6A
:106880002068C00701D01C4800E01C4821680906A8
:10689000C90E00D12021484321684905490F00D184
:1068A0000821F9F739FD21684903890FC84010BD57
:1068B0000C10024080B50F4881688906490F491EB7
:1068C00003290AD80C48C0467944097949008F4405
:1068D00009010A0DFFF7D2FF80BD0068C004810FD7
:1068E0000648C84080BD7D20000280BD0120C00355
:1068F00080BDC0460010024000127A000024F4005F
:10690000B0B50446384DCA2028605320286000F0F6
:1069100017F8002801D004200EE0A0782178490360
:106920000818617809020143E07800040843294609
:106930002039086000F020F800212960B0BDC04671
:1069400070B519480568194E30680024400610D407
:1069500030688021014331607D20C1002846F9F76D
:10696000DBFC681AC0433168490602D4401CFAD3E4
:106970000424204670BDC046B0B50B4804680B4DDA
:1069800028688021884328607D20C1002046F9F7CF
:10699000C3FC601AC0432968490603D5401CFAD3DA
:1069A0000420B0BD0020B0BD0C0000200C28004029
:1069B000B0B504460C4DCA20286053202860FFF76C
:1069C000BFFF002801D004200BE02078000461788C
:1069D00009020818A1784018294624390860FFF7F1
:1069E000CBFF00212960B0BD24280040B0B50D4682
:1069F0000446124884420BD01148844205D0114805
:106A0000844202D01048844215D1FFF717FF01E0FD
:106A1000FFF724FF21680904C90F8840690840185E
:106A20002946F9F779FC01461039084A914202D803
:106A3000E0600020B0BD0120B0BDC046003801407C
:106A400000440040004C004000480040EFFF0000C0
:106A5000B0B501231A0304689443CA682243026054
:106A6000032214034568A5430C692C434460DB03EF
:106A700004689C434B682343036003680C24A343CE
:106A80000C681C430460530204689C434B69234315
:106A900003601202836893438A691A43826089689B
:106AA000FFF7A4FFB0BD0000B0B51C480168022587
:106AB00029430124A143016021052046FBF786FEFE
:106AC00017484168174A0A40174951184160220681
:106AD000014608390B6813430B600A689201FCD524
:106AE000210442680A434260016829430522914318
:106AF0000160016838220A40102AFAD107210A02EF
:106B00000368934303600A03036893430360090423
:106B100002688A430260FBF735F9B0BD00200240ED
:106B20000810024006F8F9FF61010200F8B51646A8
:106B30000D4604461F4F002804D11F481F493A46FE
:106B4000FDF768FB002D04D17A1C1DA01B49FDF741
:106B500061FB1D4F3868002805D11648821C1B4870
:106B60001649FDF757FBE069002805D11148C21C02
:106B700017A01249FDF74EFBA169002901D020465C
:106B80008847072026616061102220462946FEF7CB
:106B90002FFC3437F9F7AEFA39463F68002FFBD1A6
:106BA00022462C320A600025E562F9F7A7FA28464A
:106BB000F8BDC04613050000EA85000819860008E4
:106BC0006E616D6500000000201E0020F685000843
:106BD0006261636B656E642D3E6F757470757400D1
:106BE00080B500F0FFF904480449C16104A1012205
:106BF000FFF79CFF002080BD08070020096C0008FB
:106C0000636F6E736F6C650080B50298FDF78AFC48
:106C100080BD0000F0B587B00293174604460125F9
:106C20002E020028069105D152A054493246FDF7A4
:106C3000F1FA0699082904D3721C51484F49FDF70F
:106C4000E9FA0C98002F039005D1B21C4D484B492E
:106C5000FDF7E0FA03980197002804D1F21C4A4896
:106C60004649FDF7D7FA04960D980090474E00204C
:106C7000059030604648FEF7B4FB7060A627069981
:106C8000CF402F40306810D10D462118414A00F006
:106C9000C9F9316808183060A9003F4A52582118D4
:106CA00000F0C0F93168081830605B2121542018C9
:106CB000451CFFF729F80146284600F0D7F931684E
:106CC000401800195D224270059A82706018FEF724
:106CD00088FB3168081830602118304A304DA847C9
:106CE0003168081830602118069A92002DA39A582E
:106CF000A8473168081830602118019AA847316800
:106D00000818306021182F4AA847316809183160E7
:106D10006018049D691A039A009BFFF7F9F9014670
:106D2000306840186A1C904200D30498002900DAA9
:106D30000498306071680A18FC3A234B9A4202D8D2
:106D4000FB20401A30600299002906D02118104A11
:106D500000F068F9316808183060002F06D121185A
:106D60001AA200F05FF931680818306005992154C3
:106D700007B0F0BD6C6F675F627566000B86000838
:106D8000D2850008F285000847860008940100209B
:106D9000C0850008E785000888730008827800082D
:106DA00025700008C38500080000000000000000F6
:106DB000C9850008CF85000800000000CC850008C8
:106DC000C685000881780008FEFEFFFF1B5B306D62
:106DD00000000000F0B58DB0099317460A910290AB
:106DE000FEF7FFFA04466B480068002804D16A48A1
:106DF0006AA16E4AFDF70EFAFCF752F80546FDF758
:106E000067F8083403942C460120000206900026FF
:106E10000496354608940998854200D3B5E0002DC4
:106E200008D0039804994618202120463246FDF7E1
:106E3000B5FD2DE05B20A05508988419601C0790D3
:106E4000FEF762FF0146079800F010F93018089924
:106E500040185D214170202181700021C1702046C1
:106E6000FEF7BFFA0490841908980119204650A231
:106E7000514EB0472418089801192046029AB0478D
:106E800024180898011920464C4AB0472618089C37
:106E90000A9828180590401E0090A019069C2146CB
:106EA00047A22B46FEF792FAA04200D8841900268A
:106EB0000A98B04221D0A8190999884206D2BB5D30
:106EC0000BA8082142A2FEF781FA04E00BA80822D1
:106ED0003EA1FEF78DFA089801190BAA204600F092
:106EE000A1F80419761C7007E2D108980119204610
:106EF000394A00F097F80419DAE70797089801195A
:106F0000204636A200F08EF8041900270A98B842ED
:106F100019D0E8190999884213D20798C35D184619
:106F200020385F2800D32E230BAE082130462CA238
:106F3000FEF74CFA089801192046324600F072F824
:106F400004197F1CE2E7874E3046FEF74AFA001923
:106F50000699884204D93046FEF743FA06990C1A7E
:106F6000089D29192046324600F05CF806192C4687
:106F70000021A9550096072001222B46FBF75EFC55
:106F8000079F0A983F18059D45E7FCF7BBFF0DB02A
:106F9000F0BDC046201E0020F6850008756C6F67A6
:106FA0005F68657864756D7000000000E60200009F
:106FB000442F4845582000002570000881780008BB
:106FC000253034582D253034583A20002020200018
:106FD0002530325820000000827800082020000070
:106FE00025630000B0B5084D286800280AD128465E
:106FF000083006A101242246FDF7F2FC0020686358
:107000002C606C600020B0BD201E0020756C6F6786
:10701000000000001CB504AC0194009400F046F898
:107020001CBD000070B514460D460646002904D16B
:107030000BA00C499222FDF7EDF8002C04D10AA018
:1070400008499322FDF7E6F80020215C002905D0CD
:107050003218FF2A02D82954401CF6E770BDC046FA
:10706000647374005B86000873726300F8B50E46A3
:10707000054600240A2730463946F9F74DF94743BB
:10708000F11B30220A432A55641C092E0646F1D80A
:1070900000202855611E884206D22A5C6B5C2B5466
:1070A0006A54491E401CF6E72046F8BDF0B585B08D
:1070B0001F4604920C4606468D208500002904D107
:1070C000224823492A46FDF7A5F8002F04D16A1C5F
:1070D00020481F49FDF79EF8082E04D3EA1C1E48DD
:1070E0001B49FDF797F81D48006800282BD00A9D22
:1070F000FBF7D6FE0390FCF7EBFE19490878012850
:107100000AD138462946FDF717FB0498012818D103
:107110001448FDF711FB14E0012008700097019559
:10712000039F384631462246049BFFF773FD0090CB
:107130000025304621462A463B46FBF77FFB0848A0
:107140000570FCF7DFFE05B0F0BDC046F285000813
:107150004E86000847860008D2850008201E0020C1
:1071600064200020C0850008B0B5104804681049AC
:107170002046F9F7D1F80F4D68607D20C100204608
:10718000F9F7CAF82860EFF31084EFF3108072B6B5
:10719000FBF796FE084DE961A861FBF791FEE969EE
:1071A000A969401A286084F31088B0BD0C00002043
:1071B00040420F0004000020A001002080B5FEF72F
:1071C000AFF8002080BD000000487047000000209C
:1071D00002E008C8121F08C1002AFAD170477047A0
:1071E000002001E001C1121F002AFBD170470040BE
:1071F000404040404040404041414141414040408A
:1072000040404040404040404040404040404005B9
:107210000202020202020202020202020202022030
:107220002020202020202020200202020202020230
:10723000909090909090101010101010101010104E
:107240001010101010101010101002020202020292
:1072500088888888888808080808080808080808AE
:107260000808080808080808080802020202400086
:10727000EF710008000000000000545452205245F5
:1072800047474553000000010002000100030001D0
:1072900000020001000400010002000100030001DF
:1072A00000020001000500010002000100030001CE
:1072B00000020001000400010002000100030001BF
:1072C00000020001000600010002000100030001AD
:1072D000000200010004000100020001000300019F
:1072E000000200010005000100020001000300018E
:1072F000000200010004000100020001000300017F
:10730000000200010007000100020001000300016B
:10731000000200010004000100020001000300015E
:10732000000200010005000100020001000300014D
:10733000000200010004000100020001000300013E
:10734000000200010006000100020001000300012C
:10735000000200010004000100020001000300011E
:10736000000200010005000100020001000300010D
:1073700000020001000400010002000100030001FE
:107380000002000100000000078600080000000065
:10739000000000009F78000803860008000000003D
:1073A000A7780008000000000100000002000000B3
:1073B0000400000008000000100000002000000091
:1073C00040000000800000000001000180008000FB
:1073D000800080000100030302020202017B787634
:1073E0007472707E00F6000800F0000800EC0008DF
:1073F00000E8000800E4000800E0000800FC0008C5
:107400005F5F636D645F53797374656D5F5265731D
:107410006574002253797374656D5F52657365748A
:1074200022005F5F636D645F4253505F5274635F1D
:107430004461746554696D655F436667002220424C
:107440004344E6A0BCE5BC8FE8BE93E585A5205289
:107450005443E697A5E69C9FE697B6E997B4E9857D
:107460008DE7BDAE3A792C6D2C642C682C6D2C7395
:107470002C772022005F5F636D645F544553545F37
:10748000466C6173685F57726974655F5265636FBC
:1074900072640022544553545F466C6173685F57B1
:1074A000726974655F5265636F726422005F5F6327
:1074B0006D645F544553545F466C6173685F5265F9
:1074C00061645F5265636F72640022544553545F78
:1074D000466C6173685F526561645F5265636F7289
:1074E00064220068656C6C6F007361792068656C5C
:1074F0006C6F20776F726C640076657273696F6E63
:107500000073686F772052542D546872656164204F
:1075100076657273696F6E20696E666F726D6174E5
:10752000696F6E005F5F636D645F76657273696F2C
:107530006E0073686F772052542D546872656164D1
:107540002076657273696F6E20696E666F726D6109
:1075500074696F6E006C6973745F746872656164DE
:10756000006C69737420746872656164005F5F63A6
:107570006D645F6C6973745F746872656164006CDC
:1075800069737420746872656164006C6973745FF8
:1075900073656D006C6973742073656D6170686FDD
:1075A000726520696E2073797374656D005F5F6327
:1075B0006D645F6C6973745F73656D006C6973747F
:1075C0002073656D6170686F726520696E207379D4
:1075D0007374656D006C6973745F6576656E7400B5
:1075E0006C697374206576656E7420696E2073799A
:1075F0007374656D005F5F636D645F6C6973745F66
:107600006576656E74006C697374206576656E745A
:1076100020696E2073797374656D006C6973745F93
:107620006D75746578006C697374206D7574657818
:1076300020696E2073797374656D005F5F636D649C
:107640005F6C6973745F6D75746578006C697374D1
:10765000206D7574657820696E2073797374656D1B
:10766000006C6973745F6D61696C626F78006C693E
:107670007374206D61696C20626F7820696E20736D
:10768000797374656D005F5F636D645F6C697374BB
:107690005F6D61696C626F78006C697374206D61F5
:1076A000696C20626F7820696E2073797374656DE0
:1076B000006C6973745F6D73677175657565006CD7
:1076C000697374206D657373616765207175657585
:1076D0006520696E2073797374656D005F5F636DFB
:1076E000645F6C6973745F6D736771756575650050
:1076F0006C697374206D657373616765207175655E
:10770000756520696E2073797374656D006C69739B
:10771000745F74696D6572006C6973742074696D4F
:10772000657220696E2073797374656D005F5F63A5
:107730006D645F6C6973745F74696D6572006C6908
:1077400073742074696D657220696E207379737427
:10775000656D006C697374006C69737420616C6C86
:107760002073796D626F6C20696E20737973746514
:107770006D005F5F636D645F68656C700052542DCF
:10778000546872656164207368656C6C2068656C10
:10779000702E005F5F636D645F7073004C6973747B
:1077A000207468726561647320696E207468652056
:1077B00073797374656D2E005F5F636D645F6672CD
:1077C00065650053686F7720746865206D656D6F1F
:1077D000727920757361676520696E207468652011
:1077E00073797374656D2E006C6973745F6D656D6C
:1077F000006C697374206D656D6F727920757361AB
:10780000676520696E666F726D6174696F6E006B7B
:10781000416C61726D5265636F7264282564290042
:107820006B4661756C745265636F726428256429B8
:10783000006B416C61726D5263795265636F726463
:1078400028256429006B4661756C74526379526512
:10785000636F7264282564290068725F72785F73B1
:10786000656D006273705F6872006B4E756D4F6678
:107870005265636F72647300443A2000453A2000F9
:10788000493A20006273705F666C617368001B5B2D
:10789000313B33306D001B5B306D001B5B313B3384
:1078A000316D001B5B313B33326D00202025732589
:1078B0007372656164203A68725F73746172745F99
:1078C00061646472203D202523782C20696E6465F4
:1078D000785F616464723A202523782C2068725F97
:1078E0006E756D3A2025642C2068725F7061676543
:1078F0003A25642C20726561645F64617461203A8A
:1079000020202523580D0A0D0A25730020202573F9
:107910002573466C6173685F4765744D61784E7579
:107920006D28282564295F5265636F72647328256A
:1079300064292053756D5F436865636B2825235860
:107940002920213D20636865636B5F73756D282571
:107950002358292C696E6465785F61646472203AEB
:107960002523580D0A0D0A25730020202573257341
:10797000466C6173685F457261736550616765202D
:107980006661696C65640D0A0D0A25730020202567
:10799000732573466163746F727954696D652063F2
:1079A0006865636B5F73756D206572726F720D0A27
:1079B0000D0A2573002020257325734578706972A0
:1079C0006174696F6E54696D65206973206E6F74A0
:1079D000207365740D0A0D0A257300202025732578
:1079E00073466163746F727954696D6520697320A1
:1079F0006E6F74207365740D0A0D0A2573002020C4
:107A000025732573466C6173685F57726974655F8F
:107A1000282564295265636F726428256429206EC5
:107A2000756D203E3D207265636F72646564204D04
:107A30006178206E756D282564290D0A2573002054
:107A4000202573257372656164203A68725F7374D0
:107A50006172745F61646472203D202523782C205C
:107A6000696E6465785F616464723A202523782CBE
:107A70002068725F6E756D3A2025642C2068725FF5
:107A8000706167653A25642C20726561645F64618A
:107A90007461203A20202523580D0A2573002020E8
:107AA00025732573466C6173685F45726173655019
:107AB0006167655F5265636F726473206661696CAC
:107AC00065642065726173655F706167653A202542
:107AD000235820213D20202523580D0A25730020FE
:107AE000202573257377726974653A68725F7374C1
:107AF0006172745F61646472203D202523782C20BC
:107B0000696E6465785F616464723A202523782C1D
:107B10002068725F6E756D3A2025642C2068725F54
:107B2000706167653A25642C2077726974655F64BB
:107B3000617461203A202523580D0A257300202006
:107B40002573257368725F73746172745F61646416
:107B500072203D202523782C20696E6465785F6152
:107B60006464723A202523782C2068725F6E756DEC
:107B70003A2025642C2068725F706167653A25643D
:107B80002C2077726974655F64617461203A2025E6
:107B900023580D0A257300202025732573466C6138
:107BA00073685F57726974655F282564295265633D
:107BB0006F72643A253034642D253032642D2530BF
:107BC000326420253032643A253032642C206368D8
:107BD00065636B5F73756D203A202523580D0A2568
:107BE0007300202025732573496E6465785F4672A3
:107BF000616D652E68725F696E6465785F6164644B
:107C000072203D2068725F73746172745F61646496
:107C1000725B7265636F72645D202B2069202A207D
:107C2000464C4153485F504147455F425954455F78
:107C300053495A45202D2048525F5245434F5244E4
:107C40005F4652414D455F4C454E203D202523580F
:107C50000D0A257300202025732573457261736515
:107C600020506167652025640D0A257300202025BA
:107C7000732573696E646578206E756D20282564A0
:107C800029203E2041637475616C2073746F7261AA
:107C90006765206E756D2025640D0A257300202010
:107CA00025732573466C6173685F52656164204477
:107CB000617461204D69736D617463682061742023
:107CC00061646472202523582C2065787065637484
:107CD000656420256420676F742025640D0A257370
:107CE00000202025732573466C6173685F526561BF
:107CF000645F282564295265636F726428256429AE
:107D00003A253034642D253032642D253032642CF0
:107D1000253032643A253032640D0A257300202064
:107D200025732573466C6173685F526561645F46B5
:107D30006163746F727954696D653A253034642DCE
:107D4000253032642D253032642C253032643A25BA
:107D50003032640D0A257300202025732573726567
:107D60006164203A68725F73746172745F61646405
:107D70007232203D202523780D0A25730064656149
:107D800063746976617465640A00252D2A2E732058
:107D90007072692020737461747573202020202014
:107DA0002073702020202020737461636B2073691E
:107DB0007A65206D61782075736564206C656674E2
:107DC000207469636B20206572726F720A002069EB
:107DD0006E69742020200020636C6F736520200082
:107DE0002072656164792020002073757370656E60
:107DF00064002072756E6E696E67005F5F636D640C
:107E00005F0008007368656C6C20213D2052545F50
:107E10004E554C4C00256300257325730072745F2A
:107E20007468726561645F69646C655F65786375C9
:107E300074650046756E6374696F6E5B25735D20B3
:107E40007368616C6C206E6F742062652075736559
:107E50006420696E204953520A0046756E63746946
:107E60006F6E5B25735D207368616C6C206E6F7440
:107E70002062652075736564206265666F72652097
:107E80007363686564756C65722073746172740ADB
:107E90000073697A6520213D2030006D6220213D0C
:107EA0002052545F4E554C4C0073656D20213D208F
:107EB00052545F4E554C4C006D7120213D20525460
:107EC0005F4E554C4C0062756666657220213D2000
:107ED00052545F4E554C4C006576656E7420213DC2
:107EE0002052545F4E554C4C006D757465782021BE
:107EF0003D2052545F4E554C4C0076616C756520A8
:107F00003C2030783130303030550072745F657607
:107F1000656E745F73656E640072745F73656D5F28
:107F200074616B650072745F6D757465785F746100
:107F30006B650072745F6F626A6563745F67657416
:107F40005F74797065282673656D2D3E706172656A
:107F50006E742E706172656E7429203D3D205254FE
:107F60005F4F626A6563745F436C6173735F5365EF
:107F70006D6170686F72650072745F73656D5F72BA
:107F8000656C656173650072745F6D757465785FAB
:107F900072656C656173650072745F6D625F6372B8
:107FA000656174650072745F73656D5F63726561AE
:107FB00074650072745F6D715F63726561746500F2
:107FC00072745F6576656E745F6372656174650077
:107FD00072745F6D757465785F6372656174650056
:107FE00072745F6D625F64656C6574650072745F66
:107FF00073656D5F64656C6574650072745F6D7147
:108000005F64656C6574650072745F6576656E7437
:108010005F64656C6574650072745F6D7574657816
:108020005F64656C6574650072745F6F626A656336
:10803000745F6765745F7479706528266D712D3E75
:10804000706172656E742E706172656E7429203D68
:108050003D2052545F4F626A6563745F436C617385
:10806000735F4D6573736167655175657565007202
:10807000745F6D625F6465746163680072745F73DE
:10808000656D5F6465746163680072745F6D715FD4
:108090006465746163680072745F6576656E745FB1
:1080A0006465746163680072745F6D757465785F90
:1080B0006465746163680072745F6D625F636F6EA4
:1080C00074726F6C0072745F73656D5F636F6E7452
:1080D000726F6C0072745F6D715F636F6E74726F3C
:1080E0006C0072745F6576656E745F636F6E747238
:1080F0006F6C0072745F6D757465785F636F6E741A
:10810000726F6C0072745F6D625F73656E645F772F
:108110006169740072745F6D715F73656E645F771F
:108120006169740072745F73656D5F696E69740074
:1081300072745F6D715F757267656E740072745FE3
:108140006F626A6563745F6765745F7479706528D0
:10815000266576656E742D3E706172656E742E7044
:108160006172656E7429203D3D2052545F4F626AF2
:108170006563745F436C6173735F4576656E74000D
:1081800072745F6D625F726563760072745F6D71A9
:108190005F726563760072745F6576656E745F7298
:1081A0006563760072745F6F626A6563745F6765AA
:1081B000745F7479706528266D757465782D3E70CE
:1081C0006172656E742E706172656E7429203D3D1A
:1081D0002052545F4F626A6563745F436C617373CE
:1081E0005F4D757465780072745F6F626A65637461
:1081F0005F6765745F7479706528266D622D3E70C7
:108200006172656E742E706172656E7429203D3DD9
:108210002052545F4F626A6563745F436C6173738D
:108220005F4D61696C426F78002872745F7562619E
:1082300073655F7429282872745F75696E74385F7E
:1082400074202A296D656D202B2053495A454F46CD
:108250005F5354525543545F4D454D2920252052BC
:10826000545F414C49474E5F53495A45203D3D209C
:1082700030006D656D2D3E6D61676963203D3D2069
:10828000484541505F4D414749430072745F7265F4
:10829000616C6C6F630072745F6D616C6C6F630016
:1082A0002872745F75696E74385F74202A29726D44
:1082B000656D203E3D202872745F75696E74385F6D
:1082C00074202A29686561705F70747220262620E8
:1082D0002872745F75696E74385F74202A29726D14
:1082E000656D203C202872745F75696E74385F7408
:1082F000202A29686561705F656E64002872745F6A
:1083000075626173655F74296D656D202B2053491B
:108310005A454F465F5354525543545F4D454D2087
:108320002B2073697A65203C3D202872745F75624A
:108330006173655F7429686561705F656E64007262
:10834000745F6672656500706C75675F686F6C65F9
:10835000730072745F73797374656D5F68656170C3
:108360005F696E697400696E666F726D6174696FC2
:108370006E20213D2052545F4E554C4C006F626A76
:1083800065637420213D2052545F4E554C4C007261
:10839000745F6F626A6563745F66696E64007274AD
:1083A0005F6F626A6563745F616C6C6F6361746553
:1083B0000072745F6F626A6563745F64656C657494
:1083C000650072745F6F626A6563745F696E697479
:1083D0000074687265616420213D2052545F4E55DF
:1083E0004C4C0072745F6F626A6563745F6765749A
:1083F0005F74797065282872745F6F626A65637450
:108400005F742974687265616429203D3D2052546F
:108410005F4F626A6563745F436C6173735F546836
:10842000726561640072745F7468726561645F7321
:10843000757370656E640072745F746872656164F0
:108440005F726573756D650072745F7468726561E3
:10845000645F64656C6574650072745F74687265EE
:1084600061645F6465746163680072745F746872EC
:108470006561645F64656C61795F756E74696C00D9
:1084800072745F7468726561645F636F6E74726F3B
:108490006C0072745F7468726561645F736C6565AB
:1084A000700072745F7468726561645F7374617286
:1084B0007475700072745F7468726561645F696E70
:1084C00069740072745F7468726561645F74696D69
:1084D000656F75740074696D657220213D2052547A
:1084E0005F4E554C4C0072745F74696D65725F64C9
:1084F000656C6574650072745F74696D65725F6444
:1085000065746163680072745F74696D65725F633E
:108510006F6E74726F6C0072745F74696D65725FF8
:1085200073746F700072745F6F626A6563745F6703
:1085300065745F74797065282674696D65722D3E67
:10854000706172656E7429203D3D2052545F4F6208
:108550006A6563745F436C6173735F54696D6572C0
:108560000072745F74696D65725F73746172740018
:108570002020257325737374617274757020756182
:108580007274315F646D615F72785F746872656187
:10859000642072657475726E203D2025640D0A2575
:1085A000730055534152543120496E69740064720E
:1085B000765F75617274005465726D696E616C00EE
:1085C0000D0A00412F00442F00452F00492F00576E
:1085D0002F006C6576656C203C3D204C4F475F4C0E
:1085E000564C5F444247001B5B006261636B656EE3
:1085F000640074616700756C6F672E696E69745FE3
:108600006F6B0033336D0033356D00756C6F675FD2
:10861000666F726D6174657200756C6F675F626121
:10862000636B656E645F726567697374657200750C
:108630006C6F675F6261636B656E645F756E7265B8
:1086400067697374657200666F726D617400756C32
:108650006F675F766F757470757400756C6F675FA8
:1086600073747263707900005164000849640008F3
:10867000E56F00084564000851070008CD23000895
:108680006D460008E16B000891050008AD06000882
:10869000092A00085D2600084D64000800740008DF
:1086A00013740008291E0008227400083D74000895
:1086B000E10700087574000893740008A11E000803
:1086C000AD740008CA7400082D1E0008E374000889
:1086D000E9740008092F0008F97400080175000802
:1086E000BD7100082475000832750008BD710008CE
:1086F0005575000861750008C13600086D750008E1
:108700007F750008C13600088B7500089475000855
:1087100095350008AD750008BC7500089535000852
:10872000D5750008E0750008F12F0008F575000800
:1087300006760008F12F00081B7600082676000850
:10874000853400083B7600084C7600088534000824
:10875000617600086E76000895310008867600087C
:108760009976000895310008B1760008BF760008B8
:1087700051330008DC760008F07600085133000819
:108780000D77000818770008393800082D770008A1
:108790003E770008393800085377000858770008FA
:1087A000852F0008727700087D770008353E0008A5
:1087B000937700089C77000833280008B8770008F2
:1087C000C377000829280008E8770008F177000837
:1087D000E5320008F8870008000000208000000053
:1087E000D07100087888000880000020E82300008D
:1087F000E0710008219EFFFF000000000100000062
:10880000010000000024F40001000000140000201A
:10881000140000209000000002000000240000204E
:108820002400002028000000030000003400002085
:10883000340000202C000000040000004400002050
:108840004400002028000000050000005400002023
:1088500054000020380000000600000064000020E2
:1088600064000020440000000A00000074000020A2
:08887000740000203400000038
:04000005080000C12E
:00000001FF
